 mlib_image

 Timestamp is 157b64ba (reproducible build file hash)

 Preferred load address is 0000000180000000

 Start         Length     Name                   Class
 0001:00000000 0006d070H .text$mn                CODE
 0001:0006d070 00000036H .text$mn$00             CODE
 0001:0006d0a6 00000092H .text$x                 CODE
 0002:00000000 00000108H .idata$5                DATA
 0002:00000108 00000038H .00cfg                  DATA
 0002:00000140 00000008H .CRT$XCA                DATA
 0002:00000148 00000008H .CRT$XCZ                DATA
 0002:00000150 00000008H .CRT$XIA                DATA
 0002:00000158 00000008H .CRT$XIZ                DATA
 0002:00000160 00000008H .CRT$XPA                DATA
 0002:00000168 00000008H .CRT$XPZ                DATA
 0002:00000170 00000008H .CRT$XTA                DATA
 0002:00000178 00000008H .CRT$XTZ                DATA
 0002:00000180 00000000H .gehcont$y              DATA
 0002:00000180 00000000H .gfids$y                DATA
 0002:00000180 0000b680H .rdata                  DATA
 0002:0000b800 00000000H .rdata$CastGuardVftablesA DATA
 0002:0000b800 00000000H .rdata$CastGuardVftablesC DATA
 0002:0000b800 0000006cH .rdata$voltmd           DATA
 0002:0000b86c 000002bcH .rdata$zzzdbg           DATA
 0002:0000bb28 00000008H .rtc$IAA                DATA
 0002:0000bb30 00000008H .rtc$IZZ                DATA
 0002:0000bb38 00000008H .rtc$TAA                DATA
 0002:0000bb40 00000008H .rtc$TZZ                DATA
 0002:0000bb48 000029b8H .xdata                  DATA
 0002:0000e500 00000124H .edata                  DATA
 0002:0000e624 00000050H .idata$2                DATA
 0002:0000e674 00000014H .idata$3                DATA
 0002:0000e688 00000108H .idata$4                DATA
 0002:0000e790 000002ccH .idata$6                DATA
 0003:00000000 00000050H .data                   DATA
 0003:00000050 000005f8H .bss                    DATA
 0004:00000000 000016a4H .pdata                  DATA
 0005:00000000 00000060H .rsrc$01                DATA
 0005:00000060 00000320H .rsrc$02                DATA

  Address         Publics by Value              Rva+Base               Lib:Object

 0000:00000000       __AbsoluteZero             0000000000000000     <absolute>
 0000:00000000       ___safe_se_handler_count   0000000000000000     <absolute>
 0000:00000000       ___safe_se_handler_table   0000000000000000     <absolute>
 0000:00000000       __arm64x_extra_rfe_table   0000000000000000     <absolute>
 0000:00000000       __arm64x_extra_rfe_table_size 0000000000000000     <absolute>
 0000:00000000       __arm64x_native_entrypoint 0000000000000000     <absolute>
 0000:00000000       __arm64x_redirection_metadata 0000000000000000     <absolute>
 0000:00000000       __arm64x_redirection_metadata_count 0000000000000000     <absolute>
 0000:00000000       __dynamic_value_reloc_table 0000000000000000     <absolute>
 0000:00000000       __enclave_config           0000000000000000     <absolute>
 0000:00000000       __guard_check_icall_a64n_fptr 0000000000000000     <absolute>
 0000:00000000       __guard_eh_cont_count      0000000000000000     <absolute>
 0000:00000000       __guard_eh_cont_table      0000000000000000     <absolute>
 0000:00000000       __guard_fids_count         0000000000000000     <absolute>
 0000:00000000       __guard_fids_table         0000000000000000     <absolute>
 0000:00000000       __guard_iat_count          0000000000000000     <absolute>
 0000:00000000       __guard_iat_table          0000000000000000     <absolute>
 0000:00000000       __guard_longjmp_count      0000000000000000     <absolute>
 0000:00000000       __guard_longjmp_table      0000000000000000     <absolute>
 0000:00000000       __hybrid_auxiliary_delayload_iat 0000000000000000     <absolute>
 0000:00000000       __hybrid_auxiliary_delayload_iat_copy 0000000000000000     <absolute>
 0000:00000000       __hybrid_auxiliary_iat     0000000000000000     <absolute>
 0000:00000000       __hybrid_auxiliary_iat_copy 0000000000000000     <absolute>
 0000:00000000       __hybrid_code_map          0000000000000000     <absolute>
 0000:00000000       __hybrid_code_map_count    0000000000000000     <absolute>
 0000:00000000       __hybrid_image_info_bitfield 0000000000000000     <absolute>
 0000:00000000       __x64_code_ranges_to_entry_points 0000000000000000     <absolute>
 0000:00000000       __x64_code_ranges_to_entry_points_count 0000000000000000     <absolute>
 0000:00000100       __guard_flags              0000000000000100     <absolute>
 0000:00000000       __ImageBase                0000000180000000     <linker-defined>
 0001:00000000       j2d_mlib_ImageAffine       0000000180001000 f   mlib_ImageAffine.obj
 0001:00000030       mlib_ImageAffine_alltypes  0000000180001030 f   mlib_ImageAffine.obj
 0001:00000370       mlib_ImageAffineEdgeExtend_BC 0000000180001370 f   mlib_ImageAffineEdge.obj
 0001:00015530       mlib_ImageAffineEdgeExtend_BL 0000000180016530 f   mlib_ImageAffineEdge.obj
 0001:0001c130       mlib_ImageAffineEdgeNearest 000000018001d130 f   mlib_ImageAffineEdge.obj
 0001:0001d9f0       mlib_ImageAffineEdgeZero   000000018001e9f0 f   mlib_ImageAffineEdge.obj
 0001:0001e300       mlib_ImageAffine_d64_1ch_bc 000000018001f300 f   mlib_ImageAffine_BC_D64.obj
 0001:0001ecd0       mlib_ImageAffine_d64_2ch_bc 000000018001fcd0 f   mlib_ImageAffine_BC_D64.obj
 0001:0001f770       mlib_ImageAffine_d64_3ch_bc 0000000180020770 f   mlib_ImageAffine_BC_D64.obj
 0001:00020220       mlib_ImageAffine_d64_4ch_bc 0000000180021220 f   mlib_ImageAffine_BC_D64.obj
 0001:00020ce0       mlib_ImageAffine_f32_1ch_bc 0000000180021ce0 f   mlib_ImageAffine_BC_F32.obj
 0001:000216a0       mlib_ImageAffine_f32_2ch_bc 00000001800226a0 f   mlib_ImageAffine_BC_F32.obj
 0001:00022160       mlib_ImageAffine_f32_3ch_bc 0000000180023160 f   mlib_ImageAffine_BC_F32.obj
 0001:00022c20       mlib_ImageAffine_f32_4ch_bc 0000000180023c20 f   mlib_ImageAffine_BC_F32.obj
 0001:000236e0       mlib_ImageAffine_s32_1ch_bc 00000001800246e0 f   mlib_ImageAffine_BC_S32.obj
 0001:000241e0       mlib_ImageAffine_s32_2ch_bc 00000001800251e0 f   mlib_ImageAffine_BC_S32.obj
 0001:00024d80       mlib_ImageAffine_s32_3ch_bc 0000000180025d80 f   mlib_ImageAffine_BC_S32.obj
 0001:00025930       mlib_ImageAffine_s32_4ch_bc 0000000180026930 f   mlib_ImageAffine_BC_S32.obj
 0001:000264e0       mlib_ImageAffine_d64_1ch_bl 00000001800274e0 f   mlib_ImageAffine_BL_D64.obj
 0001:00026aa0       mlib_ImageAffine_d64_2ch_bl 0000000180027aa0 f   mlib_ImageAffine_BL_D64.obj
 0001:00027280       mlib_ImageAffine_d64_3ch_bl 0000000180028280 f   mlib_ImageAffine_BL_D64.obj
 0001:00027720       mlib_ImageAffine_d64_4ch_bl 0000000180028720 f   mlib_ImageAffine_BL_D64.obj
 0001:00027d10       mlib_ImageAffine_f32_1ch_bl 0000000180028d10 f   mlib_ImageAffine_BL_F32.obj
 0001:000282c0       mlib_ImageAffine_f32_2ch_bl 00000001800292c0 f   mlib_ImageAffine_BL_F32.obj
 0001:00028aa0       mlib_ImageAffine_f32_3ch_bl 0000000180029aa0 f   mlib_ImageAffine_BL_F32.obj
 0001:00028f30       mlib_ImageAffine_f32_4ch_bl 0000000180029f30 f   mlib_ImageAffine_BL_F32.obj
 0001:00029520       mlib_ImageAffine_s32_1ch_bl 000000018002a520 f   mlib_ImageAffine_BL_S32.obj
 0001:00029c30       mlib_ImageAffine_s32_2ch_bl 000000018002ac30 f   mlib_ImageAffine_BL_S32.obj
 0001:0002a680       mlib_ImageAffine_s32_3ch_bl 000000018002b680 f   mlib_ImageAffine_BL_S32.obj
 0001:0002ac60       mlib_ImageAffine_s32_4ch_bl 000000018002bc60 f   mlib_ImageAffine_BL_S32.obj
 0001:0002b3b0       mlib_ImageAffine_d64_1ch_nn 000000018002c3b0 f   mlib_ImageAffine_NN.obj
 0001:0002b5f0       mlib_ImageAffine_d64_2ch_nn 000000018002c5f0 f   mlib_ImageAffine_NN.obj
 0001:0002b870       mlib_ImageAffine_d64_3ch_nn 000000018002c870 f   mlib_ImageAffine_NN.obj
 0001:0002bb10       mlib_ImageAffine_d64_4ch_nn 000000018002cb10 f   mlib_ImageAffine_NN.obj
 0001:0002bde0       mlib_ImageAffine_s32_1ch_nn 000000018002cde0 f   mlib_ImageAffine_NN.obj
 0001:0002c140       mlib_ImageAffine_s32_2ch_nn 000000018002d140 f   mlib_ImageAffine_NN.obj
 0001:0002c3c0       mlib_ImageAffine_s32_3ch_nn 000000018002d3c0 f   mlib_ImageAffine_NN.obj
 0001:0002c660       mlib_ImageAffine_s32_4ch_nn 000000018002d660 f   mlib_ImageAffine_NN.obj
 0001:0002c920       mlib_ImageClippingMxN      000000018002d920 f   mlib_ImageClipping.obj
 0001:0002cbf0       mlib_ImageConvClearEdge_Bit 000000018002dbf0 f   mlib_ImageConvClearEdge_Bit.obj
 0001:0002d140       mlib_ImageConvClearEdge_Fp 000000018002e140 f   mlib_ImageConvClearEdge_Fp.obj
 0001:0002d540       mlib_ImageConvCopyEdge_Bit 000000018002e540 f   mlib_ImageConvCopyEdge_Bit.obj
 0001:0002e550       j2d_mlib_ImageConvKernelConvert 000000018002f550 f   mlib_ImageConvKernelConvert.obj
 0001:0002f270       j2d_mlib_ImageConvMxN      0000000180030270 f   mlib_ImageConvMxN.obj
 0001:0002f2d0       mlib_ImageConvMxN_f        00000001800302d0 f   mlib_ImageConvMxN.obj
 0001:00030920       mlib_convMxNext_d64        0000000180031920 f   mlib_ImageConvMxN_Fp.obj
 0001:00030e20       mlib_convMxNext_f32        0000000180031e20 f   mlib_ImageConvMxN_Fp.obj
 0001:000317a0       mlib_convMxNext_s32        00000001800327a0 f   mlib_ImageConvMxN_ext.obj
 0001:00032cc0       mlib_convMxNext_s16        0000000180033cc0 f   mlib_ImageConv_16ext.obj
 0001:00034f90       mlib_i_convMxNext_s16      0000000180035f90 f   mlib_ImageConv_16ext.obj
 0001:00037b30       mlib_convMxNnw_s16         0000000180038b30 f   mlib_ImageConv_16nw.obj
 0001:00039870       mlib_i_convMxNnw_s16       000000018003a870 f   mlib_ImageConv_16nw.obj
 0001:0003b730       mlib_convMxNnw_s32         000000018003c730 f   mlib_ImageConv_32nw.obj
 0001:0003e250       mlib_c_convMxNext_u8       000000018003f250 f   mlib_ImageConv_8ext.obj
 0001:00040590       mlib_i_convMxNext_u8       0000000180041590 f   mlib_ImageConv_8ext.obj
 0001:000431b0       mlib_c_convMxNnw_u8        00000001800441b0 f   mlib_ImageConv_8nw.obj
 0001:00044f70       mlib_i_convMxNnw_u8        0000000180045f70 f   mlib_ImageConv_8nw.obj
 0001:00046c30       mlib_convMxNnw_d64         0000000180047c30 f   mlib_ImageConv_D64nw.obj
 0001:00048350       mlib_convMxNnw_f32         0000000180049350 f   mlib_ImageConv_F32nw.obj
 0001:0004a2a0       mlib_convMxNext_u16        000000018004b2a0 f   mlib_ImageConv_u16ext.obj
 0001:0004c6e0       mlib_i_convMxNext_u16      000000018004d6e0 f   mlib_ImageConv_u16ext.obj
 0001:0004f330       mlib_convMxNnw_u16         0000000180050330 f   mlib_ImageConv_u16nw.obj
 0001:00051140       mlib_i_convMxNnw_u16       0000000180052140 f   mlib_ImageConv_u16nw.obj
 0001:000525e0       mlib_ImageCopy_bit_na      00000001800535e0 f   mlib_ImageCopy_Bit.obj
 0001:000527a0       j2d_mlib_ImageCreate       00000001800537a0 f   mlib_ImageCreate.obj
 0001:00052970       j2d_mlib_ImageCreateStruct 0000000180053970 f   mlib_ImageCreate.obj
 0001:00052a10       j2d_mlib_ImageDelete       0000000180053a10 f   mlib_ImageCreate.obj
 0001:00052a60       mlib_ImageSet              0000000180053a60 f   mlib_ImageCreate.obj
 0001:00052c40       mlib_ImageSetSubimage      0000000180053c40 f   mlib_ImageCreate.obj
 0001:00052d70       mlib_ImageLookUpSI_S16_D64 0000000180053d70 f   mlib_ImageLookUp_64.obj
 0001:000530a0       mlib_ImageLookUpSI_S32_D64 00000001800540a0 f   mlib_ImageLookUp_64.obj
 0001:000533d0       mlib_ImageLookUpSI_U16_D64 00000001800543d0 f   mlib_ImageLookUp_64.obj
 0001:00053650       mlib_ImageLookUpSI_U8_D64  0000000180054650 f   mlib_ImageLookUp_64.obj
 0001:00054260       mlib_ImageLookUp_S16_D64   0000000180055260 f   mlib_ImageLookUp_64.obj
 0001:00054610       mlib_ImageLookUp_S32_D64   0000000180055610 f   mlib_ImageLookUp_64.obj
 0001:000549c0       mlib_ImageLookUp_U16_D64   00000001800559c0 f   mlib_ImageLookUp_64.obj
 0001:00054cb0       mlib_ImageLookUp_U8_D64    0000000180055cb0 f   mlib_ImageLookUp_64.obj
 0001:00055810       mlib_ImageLookUp_Bit_U8_1  0000000180056810 f   mlib_ImageLookUp_Bit.obj
 0001:00055b90       mlib_ImageLookUp_Bit_U8_2  0000000180056b90 f   mlib_ImageLookUp_Bit.obj
 0001:00055e30       mlib_ImageLookUp_Bit_U8_3  0000000180056e30 f   mlib_ImageLookUp_Bit.obj
 0001:000564a0       mlib_ImageLookUp_Bit_U8_4  00000001800574a0 f   mlib_ImageLookUp_Bit.obj
 0001:000567f0       mlib_AffineEdges           00000001800577f0 f   mlib_ImageScanPoly.obj
 0001:000579a0       mlib_ilogb                 00000001800589a0 f   mlib_ImageUtils.obj
 0001:00057a10       mlib_ImageAffine_u8_1ch_bc 0000000180058a10 f   mlib_c_ImageAffine_BC.obj
 0001:00057f30       mlib_ImageAffine_u8_2ch_bc 0000000180058f30 f   mlib_c_ImageAffine_BC.obj
 0001:00058510       mlib_ImageAffine_u8_3ch_bc 0000000180059510 f   mlib_c_ImageAffine_BC.obj
 0001:00058af0       mlib_ImageAffine_u8_4ch_bc 0000000180059af0 f   mlib_c_ImageAffine_BC.obj
 0001:000590e0       mlib_ImageAffine_s16_1ch_bc 000000018005a0e0 f   mlib_c_ImageAffine_BC_S16.obj
 0001:00059610       mlib_ImageAffine_s16_2ch_bc 000000018005a610 f   mlib_c_ImageAffine_BC_S16.obj
 0001:00059c20       mlib_ImageAffine_s16_3ch_bc 000000018005ac20 f   mlib_c_ImageAffine_BC_S16.obj
 0001:0005a230       mlib_ImageAffine_s16_4ch_bc 000000018005b230 f   mlib_c_ImageAffine_BC_S16.obj
 0001:0005a850       mlib_ImageAffine_u16_1ch_bc 000000018005b850 f   mlib_c_ImageAffine_BC_U16.obj
 0001:0005ada0       mlib_ImageAffine_u16_2ch_bc 000000018005bda0 f   mlib_c_ImageAffine_BC_U16.obj
 0001:0005b3f0       mlib_ImageAffine_u16_3ch_bc 000000018005c3f0 f   mlib_c_ImageAffine_BC_U16.obj
 0001:0005ba40       mlib_ImageAffine_u16_4ch_bc 000000018005ca40 f   mlib_c_ImageAffine_BC_U16.obj
 0001:0005c0a0       mlib_ImageAffine_u8_1ch_bl 000000018005d0a0 f   mlib_c_ImageAffine_BL.obj
 0001:0005c330       mlib_ImageAffine_u8_2ch_bl 000000018005d330 f   mlib_c_ImageAffine_BL.obj
 0001:0005c700       mlib_ImageAffine_u8_3ch_bl 000000018005d700 f   mlib_c_ImageAffine_BL.obj
 0001:0005cb70       mlib_ImageAffine_u8_4ch_bl 000000018005db70 f   mlib_c_ImageAffine_BL.obj
 0001:0005d0f0       mlib_ImageAffine_s16_1ch_bl 000000018005e0f0 f   mlib_c_ImageAffine_BL_S16.obj
 0001:0005d3b0       mlib_ImageAffine_s16_2ch_bl 000000018005e3b0 f   mlib_c_ImageAffine_BL_S16.obj
 0001:0005d7a0       mlib_ImageAffine_s16_3ch_bl 000000018005e7a0 f   mlib_c_ImageAffine_BL_S16.obj
 0001:0005dc60       mlib_ImageAffine_s16_4ch_bl 000000018005ec60 f   mlib_c_ImageAffine_BL_S16.obj
 0001:0005e220       mlib_ImageAffine_u16_1ch_bl 000000018005f220 f   mlib_c_ImageAffine_BL_U16.obj
 0001:0005e4e0       mlib_ImageAffine_u16_2ch_bl 000000018005f4e0 f   mlib_c_ImageAffine_BL_U16.obj
 0001:0005e8d0       mlib_ImageAffine_u16_3ch_bl 000000018005f8d0 f   mlib_c_ImageAffine_BL_U16.obj
 0001:0005ed90       mlib_ImageAffine_u16_4ch_bl 000000018005fd90 f   mlib_c_ImageAffine_BL_U16.obj
 0001:0005f350       mlib_ImageAffine_s16_1ch_nn 0000000180060350 f   mlib_c_ImageAffine_NN.obj
 0001:0005f4c0       mlib_ImageAffine_s16_2ch_nn 00000001800604c0 f   mlib_c_ImageAffine_NN.obj
 0001:0005f690       mlib_ImageAffine_s16_3ch_nn 0000000180060690 f   mlib_c_ImageAffine_NN.obj
 0001:0005f890       mlib_ImageAffine_s16_4ch_nn 0000000180060890 f   mlib_c_ImageAffine_NN.obj
 0001:0005fad0       mlib_ImageAffine_u8_1ch_nn 0000000180060ad0 f   mlib_c_ImageAffine_NN.obj
 0001:0005fbd0       mlib_ImageAffine_u8_2ch_nn 0000000180060bd0 f   mlib_c_ImageAffine_NN.obj
 0001:0005fd80       mlib_ImageAffine_u8_3ch_nn 0000000180060d80 f   mlib_c_ImageAffine_NN.obj
 0001:0005ff70       mlib_ImageAffine_u8_4ch_nn 0000000180060f70 f   mlib_c_ImageAffine_NN.obj
 0001:000601b0       mlib_ImageConvClearEdge    00000001800611b0 f   mlib_c_ImageConvClearEdge.obj
 0001:000608b0       mlib_ImageConvZeroEdge     00000001800618b0 f   mlib_c_ImageConvClearEdge.obj
 0001:00060930       mlib_ImageConvCopyEdge     0000000180061930 f   mlib_c_ImageConvCopyEdge.obj
 0001:00061dc0       mlib_ImageConvVersion      0000000180062dc0 f   mlib_c_ImageConvVersion.obj
 0001:00061e60       mlib_convMxNext_u8         0000000180062e60 f   mlib_c_ImageConv_f.obj
 0001:00061f20       mlib_convMxNnw_u8          0000000180062f20 f   mlib_c_ImageConv_f.obj
 0001:00061fd0       mlib_ImageCopy_na          0000000180062fd0 f   mlib_c_ImageCopy.obj
 0001:000621f0       j2d_mlib_ImageLookUp       00000001800631f0 f   mlib_c_ImageLookUp.obj
 0001:00062c90       mlib_c_ImageLookUpSI_S16_S16 0000000180063c90 f   mlib_c_ImageLookUp_f.obj
 0001:00062c90       mlib_c_ImageLookUpSI_S16_U16 0000000180063c90 f   mlib_c_ImageLookUp_f.obj
 0001:00062fb0       mlib_c_ImageLookUpSI_S16_S32 0000000180063fb0 f   mlib_c_ImageLookUp_f.obj
 0001:000632d0       mlib_c_ImageLookUpSI_S16_U8 00000001800642d0 f   mlib_c_ImageLookUp_f.obj
 0001:00064550       mlib_c_ImageLookUpSI_S32_S16 0000000180065550 f   mlib_c_ImageLookUp_f.obj
 0001:00064550       mlib_c_ImageLookUpSI_S32_U16 0000000180065550 f   mlib_c_ImageLookUp_f.obj
 0001:00064860       mlib_c_ImageLookUpSI_S32_S32 0000000180065860 f   mlib_c_ImageLookUp_f.obj
 0001:00064b80       mlib_c_ImageLookUpSI_S32_U8 0000000180065b80 f   mlib_c_ImageLookUp_f.obj
 0001:00064e40       mlib_c_ImageLookUpSI_U16_S16 0000000180065e40 f   mlib_c_ImageLookUp_f.obj
 0001:00064e40       mlib_c_ImageLookUpSI_U16_U16 0000000180065e40 f   mlib_c_ImageLookUp_f.obj
 0001:000650e0       mlib_c_ImageLookUpSI_U16_S32 00000001800660e0 f   mlib_c_ImageLookUp_f.obj
 0001:00065380       mlib_c_ImageLookUpSI_U16_U8 0000000180066380 f   mlib_c_ImageLookUp_f.obj
 0001:00065a90       mlib_c_ImageLookUpSI_U8_S16 0000000180066a90 f   mlib_c_ImageLookUp_f.obj
 0001:00066420       mlib_c_ImageLookUpSI_U8_S32 0000000180067420 f   mlib_c_ImageLookUp_f.obj
 0001:00066d80       mlib_c_ImageLookUpSI_U8_U8 0000000180067d80 f   mlib_c_ImageLookUp_f.obj
 0001:000677d0       mlib_c_ImageLookUp_S16_S16 00000001800687d0 f   mlib_c_ImageLookUp_f.obj
 0001:000677d0       mlib_c_ImageLookUp_S16_U16 00000001800687d0 f   mlib_c_ImageLookUp_f.obj
 0001:00067b40       mlib_c_ImageLookUp_S16_S32 0000000180068b40 f   mlib_c_ImageLookUp_f.obj
 0001:00067ef0       mlib_c_ImageLookUp_S16_U8  0000000180068ef0 f   mlib_c_ImageLookUp_f.obj
 0001:00068290       mlib_c_ImageLookUp_S32_S16 0000000180069290 f   mlib_c_ImageLookUp_f.obj
 0001:00068290       mlib_c_ImageLookUp_S32_U16 0000000180069290 f   mlib_c_ImageLookUp_f.obj
 0001:00068680       mlib_c_ImageLookUp_S32_S32 0000000180069680 f   mlib_c_ImageLookUp_f.obj
 0001:000689f0       mlib_c_ImageLookUp_S32_U8  00000001800699f0 f   mlib_c_ImageLookUp_f.obj
 0001:00068d60       mlib_c_ImageLookUp_U16_S16 0000000180069d60 f   mlib_c_ImageLookUp_f.obj
 0001:00068d60       mlib_c_ImageLookUp_U16_U16 0000000180069d60 f   mlib_c_ImageLookUp_f.obj
 0001:00069000       mlib_c_ImageLookUp_U16_S32 000000018006a000 f   mlib_c_ImageLookUp_f.obj
 0001:000692e0       mlib_c_ImageLookUp_U16_U8  000000018006a2e0 f   mlib_c_ImageLookUp_f.obj
 0001:000695b0       mlib_c_ImageLookUp_U8_S16  000000018006a5b0 f   mlib_c_ImageLookUp_f.obj
 0001:0006a790       mlib_c_ImageLookUp_U8_S32  000000018006b790 f   mlib_c_ImageLookUp_f.obj
 0001:0006b250       mlib_c_ImageLookUp_U8_U8   000000018006c250 f   mlib_c_ImageLookUp_f.obj
 0001:0006c230       mlib_free                  000000018006d230 f   mlib_sys.obj
 0001:0006c240       mlib_malloc                000000018006d240 f   mlib_sys.obj
 0001:0006c24c       __GSHandlerCheck           000000018006d24c f   MSVCRT:gshandler.obj
 0001:0006c26c       __GSHandlerCheckCommon     000000018006d26c f   MSVCRT:gshandler.obj
 0001:0006c2e0       __security_check_cookie    000000018006d2e0 f   MSVCRT:amdsecgs.obj
 0001:0006c310       __chkstk                   000000018006d310 f   MSVCRT:chkstk.obj
 0001:0006c310       _alloca_probe              000000018006d310 f   MSVCRT:chkstk.obj
 0001:0006c360       __isa_available_init       000000018006d360 f   MSVCRT:cpu_disp.obj
 0001:0006c82c       _DllMainCRTStartup         000000018006d82c f   MSVCRT:dll_dllmain.obj
 0001:0006c86c       __raise_securityfailure    000000018006d86c f   MSVCRT:gs_report.obj
 0001:0006c8a0       __report_gsfailure         000000018006d8a0 f   MSVCRT:gs_report.obj
 0001:0006c9e8       __security_init_cookie     000000018006d9e8 f   MSVCRT:gs_support.obj
 0001:0006ca94       DllMain                    000000018006da94 f   MSVCRT:dll_dllmain_stub.obj
 0001:0006cab8       ?__scrt_initialize_type_info@@YAXXZ 000000018006dab8 f   MSVCRT:tncleanup.obj
 0001:0006cac8       ?__scrt_uninitialize_type_info@@YAXXZ 000000018006dac8 f   MSVCRT:tncleanup.obj
 0001:0006cad4       __local_stdio_printf_options 000000018006dad4 f i MSVCRT:default_local_stdio_options.obj
 0001:0006cadc       __local_stdio_scanf_options 000000018006dadc f i MSVCRT:default_local_stdio_options.obj
 0001:0006cae4       __scrt_initialize_default_local_stdio_options 000000018006dae4 f   MSVCRT:default_local_stdio_options.obj
 0001:0006cb00       __scrt_acquire_startup_lock 000000018006db00 f   MSVCRT:utility.obj
 0001:0006cb3c       __scrt_dllmain_after_initialize_c 000000018006db3c f   MSVCRT:utility.obj
 0001:0006cb70       __scrt_dllmain_before_initialize_c 000000018006db70 f   MSVCRT:utility.obj
 0001:0006cb88       __scrt_dllmain_crt_thread_attach 000000018006db88 f   MSVCRT:utility.obj
 0001:0006cbb0       __scrt_dllmain_crt_thread_detach 000000018006dbb0 f   MSVCRT:utility.obj
 0001:0006cbc8       __scrt_dllmain_exception_filter 000000018006dbc8 f   MSVCRT:utility.obj
 0001:0006cc28       __scrt_dllmain_uninitialize_c 000000018006dc28 f   MSVCRT:utility.obj
 0001:0006cc58       __scrt_dllmain_uninitialize_critical 000000018006dc58 f   MSVCRT:utility.obj
 0001:0006cc6c       __scrt_initialize_crt      000000018006dc6c f   MSVCRT:utility.obj
 0001:0006ccb8       __scrt_initialize_onexit_tables 000000018006dcb8 f   MSVCRT:utility.obj
 0001:0006cd44       __scrt_is_nonwritable_in_current_image 000000018006dd44 f   MSVCRT:utility.obj
 0001:0006cddc       __scrt_release_startup_lock 000000018006dddc f   MSVCRT:utility.obj
 0001:0006ce00       __scrt_uninitialize_crt    000000018006de00 f   MSVCRT:utility.obj
 0001:0006ce2c       __scrt_get_dyn_tls_init_callback 000000018006de2c f   MSVCRT:dyn_tls_init.obj
 0001:0006ce34       __crt_debugger_hook        000000018006de34 f   MSVCRT:utility_desktop.obj
 0001:0006ce3c       __scrt_fastfail            000000018006de3c f   MSVCRT:utility_desktop.obj
 0001:0006cf88       _RTC_Initialize            000000018006df88 f   MSVCRT:initsect.obj
 0001:0006cfc4       _RTC_Terminate             000000018006dfc4 f   MSVCRT:initsect.obj
 0001:0006d000       _guard_check_icall_nop     000000018006e000 f i MSVCRT:guard_support.obj
 0001:0006d004       _get_startup_argv_mode     000000018006e004 f   MSVCRT:argv_mode.obj
 0001:0006d00c       __scrt_is_ucrt_dll_in_use  000000018006e00c f   MSVCRT:ucrt_detection.obj
 0001:0006d020       memcpy                     000000018006e020 f   vcruntime:VCRUNTIME140.dll
 0001:0006d026       memset                     000000018006e026 f   vcruntime:VCRUNTIME140.dll
 0001:0006d02c       __C_specific_handler       000000018006e02c f   vcruntime:VCRUNTIME140.dll
 0001:0006d032       __std_type_info_destroy_list 000000018006e032 f   vcruntime:VCRUNTIME140.dll
 0001:0006d038       _initterm                  000000018006e038 f   ucrt:api-ms-win-crt-runtime-l1-1-0.dll
 0001:0006d03e       _initterm_e                000000018006e03e f   ucrt:api-ms-win-crt-runtime-l1-1-0.dll
 0001:0006d044       _seh_filter_dll            000000018006e044 f   ucrt:api-ms-win-crt-runtime-l1-1-0.dll
 0001:0006d04a       _configure_narrow_argv     000000018006e04a f   ucrt:api-ms-win-crt-runtime-l1-1-0.dll
 0001:0006d050       _initialize_narrow_environment 000000018006e050 f   ucrt:api-ms-win-crt-runtime-l1-1-0.dll
 0001:0006d056       _initialize_onexit_table   000000018006e056 f   ucrt:api-ms-win-crt-runtime-l1-1-0.dll
 0001:0006d05c       _execute_onexit_table      000000018006e05c f   ucrt:api-ms-win-crt-runtime-l1-1-0.dll
 0001:0006d062       _cexit                     000000018006e062 f   ucrt:api-ms-win-crt-runtime-l1-1-0.dll
 0001:0006d068       __acrt_initialize          000000018006e068 f   MSVCRT:ucrt_stubs.obj
 0001:0006d068       __acrt_thread_attach       000000018006e068 f   MSVCRT:ucrt_stubs.obj
 0001:0006d068       __acrt_thread_detach       000000018006e068 f   MSVCRT:ucrt_stubs.obj
 0001:0006d068       __acrt_uninitialize        000000018006e068 f   MSVCRT:ucrt_stubs.obj
 0001:0006d068       __acrt_uninitialize_critical 000000018006e068 f   MSVCRT:ucrt_stubs.obj
 0001:0006d068       __scrt_stub_for_acrt_initialize 000000018006e068 f   MSVCRT:ucrt_stubs.obj
 0001:0006d068       __scrt_stub_for_acrt_thread_attach 000000018006e068 f   MSVCRT:ucrt_stubs.obj
 0001:0006d068       __scrt_stub_for_acrt_thread_detach 000000018006e068 f   MSVCRT:ucrt_stubs.obj
 0001:0006d068       __scrt_stub_for_acrt_uninitialize 000000018006e068 f   MSVCRT:ucrt_stubs.obj
 0001:0006d068       __scrt_stub_for_acrt_uninitialize_critical 000000018006e068 f   MSVCRT:ucrt_stubs.obj
 0001:0006d068       __vcrt_initialize          000000018006e068 f   MSVCRT:ucrt_stubs.obj
 0001:0006d068       __vcrt_thread_attach       000000018006e068 f   MSVCRT:ucrt_stubs.obj
 0001:0006d068       __vcrt_thread_detach       000000018006e068 f   MSVCRT:ucrt_stubs.obj
 0001:0006d068       __vcrt_uninitialize        000000018006e068 f   MSVCRT:ucrt_stubs.obj
 0001:0006d068       __vcrt_uninitialize_critical 000000018006e068 f   MSVCRT:ucrt_stubs.obj
 0001:0006d06c       __scrt_stub_for_is_c_termination_complete 000000018006e06c f   MSVCRT:ucrt_stubs.obj
 0001:0006d06c       _is_c_termination_complete 000000018006e06c f   MSVCRT:ucrt_stubs.obj
 0001:0006d080       _guard_dispatch_icall_nop  000000018006e080 f   MSVCRT:guard_dispatch.obj
 0001:0006d0a0       _guard_xfg_dispatch_icall_nop 000000018006e0a0 f   MSVCRT:guard_xfg_dispatch.obj
 0002:00000000       __imp_RtlCaptureContext    000000018006f000     kernel32:KERNEL32.dll
 0002:00000008       __imp_RtlLookupFunctionEntry 000000018006f008     kernel32:KERNEL32.dll
 0002:00000010       __imp_RtlVirtualUnwind     000000018006f010     kernel32:KERNEL32.dll
 0002:00000018       __imp_UnhandledExceptionFilter 000000018006f018     kernel32:KERNEL32.dll
 0002:00000020       __imp_SetUnhandledExceptionFilter 000000018006f020     kernel32:KERNEL32.dll
 0002:00000028       __imp_GetCurrentProcess    000000018006f028     kernel32:KERNEL32.dll
 0002:00000030       __imp_TerminateProcess     000000018006f030     kernel32:KERNEL32.dll
 0002:00000038       __imp_IsProcessorFeaturePresent 000000018006f038     kernel32:KERNEL32.dll
 0002:00000040       __imp_QueryPerformanceCounter 000000018006f040     kernel32:KERNEL32.dll
 0002:00000048       __imp_GetCurrentProcessId  000000018006f048     kernel32:KERNEL32.dll
 0002:00000050       __imp_GetCurrentThreadId   000000018006f050     kernel32:KERNEL32.dll
 0002:00000058       __imp_GetSystemTimeAsFileTime 000000018006f058     kernel32:KERNEL32.dll
 0002:00000060       __imp_DisableThreadLibraryCalls 000000018006f060     kernel32:KERNEL32.dll
 0002:00000068       __imp_InitializeSListHead  000000018006f068     kernel32:KERNEL32.dll
 0002:00000070       __imp_IsDebuggerPresent    000000018006f070     kernel32:KERNEL32.dll
 0002:00000078       \177KERNEL32_NULL_THUNK_DATA 000000018006f078     kernel32:KERNEL32.dll
 0002:00000080       __imp_memcpy               000000018006f080     vcruntime:VCRUNTIME140.dll
 0002:00000088       __imp_memset               000000018006f088     vcruntime:VCRUNTIME140.dll
 0002:00000090       __imp___C_specific_handler 000000018006f090     vcruntime:VCRUNTIME140.dll
 0002:00000098       __imp___std_type_info_destroy_list 000000018006f098     vcruntime:VCRUNTIME140.dll
 0002:000000a0       \177VCRUNTIME140_NULL_THUNK_DATA 000000018006f0a0     vcruntime:VCRUNTIME140.dll
 0002:000000a8       __imp_malloc               000000018006f0a8     ucrt:api-ms-win-crt-heap-l1-1-0.dll
 0002:000000b0       __imp_free                 000000018006f0b0     ucrt:api-ms-win-crt-heap-l1-1-0.dll
 0002:000000b8       \177api-ms-win-crt-heap-l1-1-0_NULL_THUNK_DATA 000000018006f0b8     ucrt:api-ms-win-crt-heap-l1-1-0.dll
 0002:000000c0       __imp__seh_filter_dll      000000018006f0c0     ucrt:api-ms-win-crt-runtime-l1-1-0.dll
 0002:000000c8       __imp__configure_narrow_argv 000000018006f0c8     ucrt:api-ms-win-crt-runtime-l1-1-0.dll
 0002:000000d0       __imp__initterm_e          000000018006f0d0     ucrt:api-ms-win-crt-runtime-l1-1-0.dll
 0002:000000d8       __imp__initialize_onexit_table 000000018006f0d8     ucrt:api-ms-win-crt-runtime-l1-1-0.dll
 0002:000000e0       __imp__execute_onexit_table 000000018006f0e0     ucrt:api-ms-win-crt-runtime-l1-1-0.dll
 0002:000000e8       __imp__cexit               000000018006f0e8     ucrt:api-ms-win-crt-runtime-l1-1-0.dll
 0002:000000f0       __imp__initterm            000000018006f0f0     ucrt:api-ms-win-crt-runtime-l1-1-0.dll
 0002:000000f8       __imp__initialize_narrow_environment 000000018006f0f8     ucrt:api-ms-win-crt-runtime-l1-1-0.dll
 0002:00000100       \177api-ms-win-crt-runtime-l1-1-0_NULL_THUNK_DATA 000000018006f100     ucrt:api-ms-win-crt-runtime-l1-1-0.dll
 0002:00000108       __guard_check_icall_fptr   000000018006f108     MSVCRT:guard_support.obj
 0002:00000110       __guard_xfg_check_icall_fptr 000000018006f110     MSVCRT:guard_support.obj
 0002:00000118       __guard_dispatch_icall_fptr 000000018006f118     MSVCRT:guard_support.obj
 0002:00000120       __guard_xfg_dispatch_icall_fptr 000000018006f120     MSVCRT:guard_support.obj
 0002:00000128       __guard_xfg_table_dispatch_icall_fptr 000000018006f128     MSVCRT:guard_support.obj
 0002:00000130       __castguard_check_failure_os_handled_fptr 000000018006f130     MSVCRT:guard_support.obj
 0002:00000138       __guard_memcpy_fptr        000000018006f138     vcruntime:softmemtag.obj
 0002:00000140       __xc_a                     000000018006f140     MSVCRT:initializers.obj
 0002:00000148       __xc_z                     000000018006f148     MSVCRT:initializers.obj
 0002:00000150       __xi_a                     000000018006f150     MSVCRT:initializers.obj
 0002:00000158       __xi_z                     000000018006f158     MSVCRT:initializers.obj
 0002:00000160       __xp_a                     000000018006f160     MSVCRT:initializers.obj
 0002:00000168       __xp_z                     000000018006f168     MSVCRT:initializers.obj
 0002:00000170       __xt_a                     000000018006f170     MSVCRT:initializers.obj
 0002:00000178       __xt_z                     000000018006f178     MSVCRT:initializers.obj
 0002:00000180       mlib_AffineFunArr_nn       000000018006f180     mlib_ImageAffine.obj
 0002:00000200       mlib_AffineFunArr_bl       000000018006f200     mlib_ImageAffine.obj
 0002:000002c0       mlib_AffineFunArr_bc       000000018006f2c0     mlib_ImageAffine.obj
 0002:00000380       __real@3ef0000000000000    000000018006f380     mlib_ImageAffineEdge.obj
 0002:00000388       __real@3fe0000000000000    000000018006f388     mlib_ImageAffineEdge.obj
 0002:00000390       __real@3ff0000000000000    000000018006f390     mlib_ImageAffineEdge.obj
 0002:00000398       __real@4004000000000000    000000018006f398     mlib_ImageAffineEdge.obj
 0002:000003a0       __real@4008000000000000    000000018006f3a0     mlib_ImageAffineEdge.obj
 0002:000003a8       __real@41dfe00000000000    000000018006f3a8     mlib_ImageAffineEdge.obj
 0002:000003b0       __real@41dfffe000000000    000000018006f3b0     mlib_ImageAffineEdge.obj
 0002:000003b8       __real@41dfffffffc00000    000000018006f3b8     mlib_ImageAffineEdge.obj
 0002:000003c0       __real@c1e0000000000000    000000018006f3c0     mlib_ImageAffineEdge.obj
 0002:000003c8       __real@37800000            000000018006f3c8     mlib_ImageAffine_BC_F32.obj
 0002:000003cc       __real@3f000000            000000018006f3cc     mlib_ImageAffine_BC_F32.obj
 0002:000003d0       __real@3f800000            000000018006f3d0     mlib_ImageAffine_BC_F32.obj
 0002:000003d4       __real@40200000            000000018006f3d4     mlib_ImageAffine_BC_F32.obj
 0002:000003d8       __real@40400000            000000018006f3d8     mlib_ImageAffine_BC_F32.obj
 0002:000003e0       __real@41d0000000000000    000000018006f3e0     mlib_ImageConvKernelConvert.obj
 0002:000003f0       __xmm@41dfffffffc0000041dfffffffc00000 000000018006f3f0     mlib_ImageConvKernelConvert.obj
 0002:00000400       __xmm@7fffffffffffffff7fffffffffffffff 000000018006f400     mlib_ImageConvKernelConvert.obj
 0002:00000410       __xmm@c1e0000000000000c1e0000000000000 000000018006f410     mlib_ImageConvKernelConvert.obj
 0002:00000420       __real@3e10000000000000    000000018006f420     mlib_ImageConvMxN_ext.obj
 0002:00000428       __real@3f10000000000000    000000018006f428     mlib_ImageConv_16ext.obj
 0002:00000430       __real@40f0000000000000    000000018006f430     mlib_ImageConv_16ext.obj
 0002:00000440       __xmm@00000003000000020000000100000000 000000018006f440     mlib_ImageConv_16ext.obj
 0002:00000450       __real@3f90000000000000    000000018006f450     mlib_ImageConv_8ext.obj
 0002:00000458       __real@4170000000000000    000000018006f458     mlib_ImageConv_8ext.obj
 0002:00000460       __real@41e0000000000000    000000018006f460     mlib_ImageConv_8ext.obj
 0002:00000470       mlib_div6_tab              000000018006f470     mlib_ImageDivTables.obj
 0002:00000670       mlib_div1_tab              000000018006f670     mlib_ImageDivTables.obj
 0002:00000870       mlib_HSL2RGB_L2            000000018006f870     mlib_ImageDivTables.obj
 0002:00000c70       mlib_HSL2RGB_F             000000018006fc70     mlib_ImageDivTables.obj
 0002:00001070       mlib_U82F32                0000000180070070     mlib_ImageDivTables.obj
 0002:00001480       mlib_U82D64                0000000180070480     mlib_ImageDivTables.obj
 0002:00001c90       mlib_FlipAndFixRotateTable 0000000180070c90     mlib_ImageDivTables.obj
 0002:00002490       mlib_filters_u8f_bc        0000000180071490     mlib_ImageFilters.obj
 0002:00003490       mlib_filters_u8f_bc2       0000000180072490     mlib_ImageFilters.obj
 0002:00004490       mlib_filters_s16f_bc       0000000180073490     mlib_ImageFilters.obj
 0002:00006490       mlib_filters_s16f_bc2      0000000180075490     mlib_ImageFilters.obj
 0002:00008490       mlib_filters_u8_bc         0000000180077490     mlib_ImageFilters.obj
 0002:00008c90       mlib_filters_u8_bc2        0000000180077c90     mlib_ImageFilters.obj
 0002:00009490       mlib_filters_s16_bc        0000000180078490     mlib_ImageFilters.obj
 0002:0000a490       mlib_filters_s16_bc2       0000000180079490     mlib_ImageFilters.obj
 0002:0000b490       __xmm@00000000000000080000000000000008 000000018007a490     mlib_ImageLookUp_64.obj
 0002:0000b4a0       __xmm@000000001fffffff000000001fffffff 000000018007a4a0     mlib_ImageLookUp_64.obj
 0002:0000b530       __real@7fefffffffffffff    000000018007a530     mlib_ImageScanPoly.obj
 0002:0000b538       __real@bfe0000000000000    000000018007a538     mlib_ImageScanPoly.obj
 0002:0000b540       __real@ffefffffffffffff    000000018007a540     mlib_ImageScanPoly.obj
 0002:0000b550       __xmm@80000000000000008000000000000000 000000018007a550     mlib_ImageScanPoly.obj
 0002:0000b560       __real@4330000000000000    000000018007a560     mlib_ImageUtils.obj
 0002:0000b568       __real@4020000000000000    000000018007a568     mlib_c_ImageConvVersion.obj
 0002:0000b570       __real@4040000000000000    000000018007a570     mlib_c_ImageConvVersion.obj
 0002:0000b578       __real@40e0000000000000    000000018007a578     mlib_c_ImageConvVersion.obj
 0002:0000b580       __xmm@00000000000000020000000000000002 000000018007a580     mlib_c_ImageLookUp_f.obj
 0002:0000b590       __xmm@00000000000000040000000000000004 000000018007a590     mlib_c_ImageLookUp_f.obj
 0002:0000b5a0       __xmm@00000000000080000000000000008000 000000018007a5a0     mlib_c_ImageLookUp_f.obj
 0002:0000b5b0       __xmm@000000003ffffffe000000003ffffffe 000000018007a5b0     mlib_c_ImageLookUp_f.obj
 0002:0000b5c0       _pDefaultRawDllMain        000000018007a5c0     MSVCRT:dll_dllmain.obj
 0002:0000b5c0       _pRawDllMain               000000018007a5c0     MSVCRT:dll_dllmain.obj
 0002:0000b5e0       __xmm@ffffffffffffffffffffffffffffffff 000000018007a5e0     MSVCRT:utility.obj
 0002:0000b5f0       _load_config_used          000000018007a5f0     MSVCRT:loadcfg.obj
 0002:0000b800       __volatile_metadata        000000018007a800     <linker-defined>
 0002:0000bb28       __rtc_iaa                  000000018007ab28     MSVCRT:initsect.obj
 0002:0000bb30       __rtc_izz                  000000018007ab30     MSVCRT:initsect.obj
 0002:0000bb38       __rtc_taa                  000000018007ab38     MSVCRT:initsect.obj
 0002:0000bb40       __rtc_tzz                  000000018007ab40     MSVCRT:initsect.obj
 0002:0000e624       __IMPORT_DESCRIPTOR_KERNEL32 000000018007d624     kernel32:KERNEL32.dll
 0002:0000e638       __IMPORT_DESCRIPTOR_VCRUNTIME140 000000018007d638     vcruntime:VCRUNTIME140.dll
 0002:0000e64c       __IMPORT_DESCRIPTOR_api-ms-win-crt-heap-l1-1-0 000000018007d64c     ucrt:api-ms-win-crt-heap-l1-1-0.dll
 0002:0000e660       __IMPORT_DESCRIPTOR_api-ms-win-crt-runtime-l1-1-0 000000018007d660     ucrt:api-ms-win-crt-runtime-l1-1-0.dll
 0002:0000e674       __NULL_IMPORT_DESCRIPTOR   000000018007d674     kernel32:KERNEL32.dll
 0003:00000000       __security_cookie_complement 000000018007e000     MSVCRT:gs_cookie.obj
 0003:00000008       __security_cookie          000000018007e008     MSVCRT:gs_cookie.obj
 0003:00000010       _fltused                   000000018007e010     MSVCRT:fltused.obj
 0003:00000020       __isa_available            000000018007e020     MSVCRT:cpu_disp.obj
 0003:00000024       __isa_enabled              000000018007e024     MSVCRT:cpu_disp.obj
 0003:00000028       __memset_fast_string_threshold 000000018007e028     MSVCRT:cpu_disp.obj
 0003:00000030       __memset_nt_threshold      000000018007e030     MSVCRT:cpu_disp.obj
 0003:00000038       __scrt_native_dllmain_reason 000000018007e038     MSVCRT:utility.obj
 0003:00000040       __scrt_ucrt_dll_is_in_use  000000018007e040     MSVCRT:ucrt_stubs.obj
 0003:00000050       __favor                    000000018007e050     MSVCRT:cpu_disp.obj
 0003:000005d0       ?__type_info_root_node@@3U__type_info_node@@A 000000018007e5d0     MSVCRT:tncleanup.obj
 0003:000005e0       ?_OptionsStorage@?1??__local_stdio_printf_options@@9@4_KA 000000018007e5e0     MSVCRT:default_local_stdio_options.obj
 0003:000005e8       ?_OptionsStorage@?1??__local_stdio_scanf_options@@9@4_KA 000000018007e5e8     MSVCRT:default_local_stdio_options.obj
 0003:000005f0       __scrt_current_native_startup_state 000000018007e5f0     MSVCRT:utility.obj
 0003:000005f8       __scrt_native_startup_lock 000000018007e5f8     MSVCRT:utility.obj
 0003:00000638       __scrt_debugger_hook_flag  000000018007e638     MSVCRT:utility_desktop.obj
 0003:00000640       __dyn_tls_init_callback    000000018007e640     <common>

 entry point at        0001:0006c82c

 Static symbols

 0000:fff7d000       .debug$S                   0000000180000000     mlib_image.exp
 0000:fff7d000       .debug$S                   0000000180000000     vcruntime:VCRUNTIME140.dll
 0000:fff7d000       .debug$S                   0000000180000000     vcruntime:VCRUNTIME140.dll
 0000:fff7d000       .debug$S                   0000000180000000     vcruntime:VCRUNTIME140.dll
 0000:fff7d000       .debug$S                   0000000180000000     vcruntime:VCRUNTIME140.dll
 0000:fff7d000       .debug$S                   0000000180000000     vcruntime:VCRUNTIME140.dll
 0000:fff7d000       .debug$S                   0000000180000000     vcruntime:VCRUNTIME140.dll
 0000:fff7d000       .debug$S                   0000000180000000     vcruntime:VCRUNTIME140.dll
 0000:fff7d000       .debug$S                   0000000180000000     ucrt:api-ms-win-crt-heap-l1-1-0.dll
 0000:fff7d000       .debug$S                   0000000180000000     ucrt:api-ms-win-crt-heap-l1-1-0.dll
 0000:fff7d000       .debug$S                   0000000180000000     ucrt:api-ms-win-crt-heap-l1-1-0.dll
 0000:fff7d000       .debug$S                   0000000180000000     ucrt:api-ms-win-crt-math-l1-1-0.dll
 0000:fff7d000       .debug$S                   0000000180000000     ucrt:api-ms-win-crt-math-l1-1-0.dll
 0002:fff91000       .idata$6                   0000000180000000     ucrt:api-ms-win-crt-math-l1-1-0.dll
 0000:fff7d000       .debug$S                   0000000180000000     ucrt:api-ms-win-crt-runtime-l1-1-0.dll
 0000:fff7d000       .debug$S                   0000000180000000     ucrt:api-ms-win-crt-runtime-l1-1-0.dll
 0000:fff7d000       .debug$S                   0000000180000000     ucrt:api-ms-win-crt-runtime-l1-1-0.dll
 0000:fff7d000       .debug$S                   0000000180000000     ucrt:api-ms-win-crt-runtime-l1-1-0.dll
 0000:fff7d000       .debug$S                   0000000180000000     ucrt:api-ms-win-crt-runtime-l1-1-0.dll
 0000:fff7d000       .debug$S                   0000000180000000     ucrt:api-ms-win-crt-runtime-l1-1-0.dll
 0000:fff7d000       .debug$S                   0000000180000000     ucrt:api-ms-win-crt-runtime-l1-1-0.dll
 0000:fff7d000       .debug$S                   0000000180000000     ucrt:api-ms-win-crt-runtime-l1-1-0.dll
 0000:fff7d000       .debug$S                   0000000180000000     ucrt:api-ms-win-crt-runtime-l1-1-0.dll
 0000:fff7d000       .debug$S                   0000000180000000     ucrt:api-ms-win-crt-runtime-l1-1-0.dll
 0000:fff7d000       .debug$S                   0000000180000000     ucrt:api-ms-win-crt-runtime-l1-1-0.dll
 0000:fff7d000       .debug$S                   0000000180000000     ucrt:api-ms-win-crt-runtime-l1-1-0.dll
 0000:fff7d000       .debug$S                   0000000180000000     kernel32:KERNEL32.dll
 0000:fff7d000       .debug$S                   0000000180000000     kernel32:KERNEL32.dll
 0000:fff7d000       .debug$S                   0000000180000000     kernel32:KERNEL32.dll
 0000:fff7d000       .debug$S                   0000000180000000     kernel32:KERNEL32.dll
 0000:fff7d000       .debug$S                   0000000180000000     kernel32:KERNEL32.dll
 0000:fff7d000       .debug$S                   0000000180000000     kernel32:KERNEL32.dll
 0000:fff7d000       .debug$S                   0000000180000000     kernel32:KERNEL32.dll
 0000:fff7d000       .debug$S                   0000000180000000     kernel32:KERNEL32.dll
 0000:fff7d000       .debug$S                   0000000180000000     kernel32:KERNEL32.dll
 0000:fff7d000       .debug$S                   0000000180000000     kernel32:KERNEL32.dll
 0000:fff7d000       .debug$S                   0000000180000000     kernel32:KERNEL32.dll
 0000:fff7d000       .debug$S                   0000000180000000     kernel32:KERNEL32.dll
 0000:fff7d000       .debug$S                   0000000180000000     kernel32:KERNEL32.dll
 0000:fff7d000       .debug$S                   0000000180000000     kernel32:KERNEL32.dll
 0000:fff7d000       .debug$S                   0000000180000000     kernel32:KERNEL32.dll
 0000:fff7d000       .debug$S                   0000000180000000     kernel32:KERNEL32.dll
 0000:fff7d000       .debug$S                   0000000180000000     kernel32:KERNEL32.dll
 0001:00015514       $LN1049                    0000000180016514     mlib_ImageAffineEdge.obj
 0001:0001c110       $LN763                     000000018001d110     mlib_ImageAffineEdge.obj
 0001:0001d9d4       $LN427                     000000018001e9d4     mlib_ImageAffineEdge.obj
 0001:0001e2e0       $LN236                     000000018001f2e0     mlib_ImageAffineEdge.obj
 0001:0002f8a4       $LN45                      00000001800308a4     mlib_ImageConvMxN.obj
 0001:0002f8bc       $LN44                      00000001800308bc     mlib_ImageConvMxN.obj
 0001:0002f8e0       mlib_ImageConvMxNMulAdd_D64 00000001800308e0 f   mlib_ImageConvMxN_Fp.obj
 0001:000300f0       mlib_ImageConvMxNMulAdd_F32 00000001800310f0 f   mlib_ImageConvMxN_Fp.obj
 0001:00031310       mlib_ImageConvMxNMulAdd_S32 0000000180032310 f   mlib_ImageConvMxN_ext.obj
 0001:00031640       mlib_ImageConvMxNS322S32_ext 0000000180032640 f   mlib_ImageConvMxN_ext.obj
 0001:00031e00       mlib_ImageConv1xN_ext      0000000180032e00 f   mlib_ImageConv_16ext.obj
 0001:00037080       mlib_ImageConv1xN          0000000180038080 f   mlib_ImageConv_16nw.obj
 0001:0003ad30       mlib_ImageConv1xN          000000018003bd30 f   mlib_ImageConv_32nw.obj
 0001:0003d380       mlib_ImageConv1xN_ext      000000018003e380 f   mlib_ImageConv_8ext.obj
 0001:00042730       mlib_ImageConv1xN          0000000180043730 f   mlib_ImageConv_8nw.obj
 0001:00046370       mlib_ImageConv1xN          0000000180047370 f   mlib_ImageConv_D64nw.obj
 0001:00047aa0       mlib_ImageConv1xN          0000000180048aa0 f   mlib_ImageConv_F32nw.obj
 0001:00049350       mlib_ImageConv1xN_ext      000000018004a350 f   mlib_ImageConv_u16ext.obj
 0001:0004e7e0       mlib_ImageConv1xN          000000018004f7e0 f   mlib_ImageConv_u16nw.obj
 0001:00052950       $LN32                      0000000180053950     mlib_ImageCreate.obj
 0001:00052c1c       $LN32                      0000000180053c1c     mlib_ImageCreate.obj
 0001:00052d4c       $LN18                      0000000180053d4c     mlib_ImageCreate.obj
 0001:00061da0       $LN340                     0000000180062da0     mlib_c_ImageConvCopyEdge.obj
 0001:0006c2d0       $$000000                   000000018006d2d0     MSVCRT:amdsecgs.obj
 0001:0006c300       $$000000                   000000018006d300     MSVCRT:chkstk.obj
 0001:0006c50c       ?dllmain_crt_dispatch@@YAHQEAUHINSTANCE__@@KQEAX@Z 000000018006d50c f   MSVCRT:dll_dllmain.obj
 0001:0006c55c       ?dllmain_crt_process_attach@@YAHQEAUHINSTANCE__@@QEAX@Z 000000018006d55c f   MSVCRT:dll_dllmain.obj
 0001:0006c674       ?dllmain_crt_process_detach@@YAH_N@Z 000000018006d674 f   MSVCRT:dll_dllmain.obj
 0001:0006c6f8       ?dllmain_dispatch@@YAHQEAUHINSTANCE__@@KQEAX@Z 000000018006d6f8 f   MSVCRT:dll_dllmain.obj
 0001:0006c974       capture_previous_context   000000018006d974 f   MSVCRT:gs_report.obj
 0001:0006d070       $$000000                   000000018006e070     MSVCRT:guard_dispatch.obj
 0001:0006d090       $$000000                   000000018006e090     MSVCRT:guard_xfg_dispatch.obj
 0001:0006d0a6       ?fin$0@?0??dllmain_crt_process_attach@@YAHQEAUHINSTANCE__@@QEAX@Z@4HA 000000018006e0a6 f   MSVCRT:dll_dllmain.obj
 0001:0006d0bd       ?fin$0@?0??dllmain_crt_process_detach@@YAH_N@Z@4HA 000000018006e0bd f   MSVCRT:dll_dllmain.obj
 0001:0006d0d6       ?fin$1@?0??dllmain_crt_process_detach@@YAH_N@Z@4HA 000000018006e0d6 f   MSVCRT:dll_dllmain.obj
 0001:0006d0ea       ?filt$0@?0??dllmain_dispatch@@YAHQEAUHINSTANCE__@@KQEAX@Z@4HA 000000018006e0ea f   MSVCRT:dll_dllmain.obj
 0001:0006d120       __scrt_is_nonwritable_in_current_image$filt$0 000000018006e120 f   MSVCRT:utility.obj
 0002:0000b4b0       mlib_bit_mask              000000018007a4b0     mlib_ImageLookUp_Bit.obj
 0002:0000b4f0       mlib_bit_mask_2            000000018007a4f0     mlib_ImageLookUp_Bit.obj
 0002:0000b500       mlib_bit_mask_3            000000018007a500     mlib_ImageLookUp_Bit.obj
 0002:0000b5c8       GS_ExceptionPointers       000000018007a5c8     MSVCRT:gs_report.obj
 0002:0000bb48       $unwind$mlib_ImageAffine_alltypes 000000018007ab48     mlib_ImageAffine.obj
 0002:0000bb68       $unwind$mlib_ImageAffineEdgeZero 000000018007ab68     mlib_ImageAffineEdge.obj
 0002:0000bb78       $chain$3$mlib_ImageAffineEdgeZero 000000018007ab78     mlib_ImageAffineEdge.obj
 0002:0000bb98       $chain$4$mlib_ImageAffineEdgeZero 000000018007ab98     mlib_ImageAffineEdge.obj
 0002:0000bba8       $unwind$mlib_ImageAffineEdgeNearest 000000018007aba8     mlib_ImageAffineEdge.obj
 0002:0000bba8       $unwind$mlib_ImageAffine_s32_1ch_bl 000000018007aba8     mlib_ImageAffine_BL_S32.obj
 0002:0000bbbc       $chain$1$mlib_ImageAffineEdgeNearest 000000018007abbc     mlib_ImageAffineEdge.obj
 0002:0000bbd4       $chain$2$mlib_ImageAffineEdgeNearest 000000018007abd4     mlib_ImageAffineEdge.obj
 0002:0000bbe4       $unwind$mlib_ImageAffineEdgeExtend_BL 000000018007abe4     mlib_ImageAffineEdge.obj
 0002:0000bbf8       $chain$6$mlib_ImageAffineEdgeExtend_BL 000000018007abf8     mlib_ImageAffineEdge.obj
 0002:0000bc24       $chain$7$mlib_ImageAffineEdgeExtend_BL 000000018007ac24     mlib_ImageAffineEdge.obj
 0002:0000bc34       $unwind$mlib_ImageAffineEdgeExtend_BC 000000018007ac34     mlib_ImageAffineEdge.obj
 0002:0000bc4c       $chain$10$mlib_ImageAffineEdgeExtend_BC 000000018007ac4c     mlib_ImageAffineEdge.obj
 0002:0000bc88       $chain$11$mlib_ImageAffineEdgeExtend_BC 000000018007ac88     mlib_ImageAffineEdge.obj
 0002:0000bc98       $chain$12$mlib_ImageAffineEdgeExtend_BC 000000018007ac98     mlib_ImageAffineEdge.obj
 0002:0000bcd4       $unwind$mlib_ImageAffine_d64_1ch_bc 000000018007acd4     mlib_ImageAffine_BC_D64.obj
 0002:0000bcd4       $unwind$mlib_ImageAffine_s32_1ch_bc 000000018007acd4     mlib_ImageAffine_BC_S32.obj
 0002:0000bce8       $chain$11$mlib_ImageAffine_d64_1ch_bc 000000018007ace8     mlib_ImageAffine_BC_D64.obj
 0002:0000bd28       $chain$12$mlib_ImageAffine_d64_1ch_bc 000000018007ad28     mlib_ImageAffine_BC_D64.obj
 0002:0000bd38       $unwind$mlib_ImageAffine_d64_2ch_bc 000000018007ad38     mlib_ImageAffine_BC_D64.obj
 0002:0000bd38       $unwind$mlib_ImageAffine_d64_3ch_bc 000000018007ad38     mlib_ImageAffine_BC_D64.obj
 0002:0000bd38       $unwind$mlib_ImageAffine_d64_4ch_bc 000000018007ad38     mlib_ImageAffine_BC_D64.obj
 0002:0000bd50       $chain$10$mlib_ImageAffine_d64_2ch_bc 000000018007ad50     mlib_ImageAffine_BC_D64.obj
 0002:0000bd8c       $chain$11$mlib_ImageAffine_d64_2ch_bc 000000018007ad8c     mlib_ImageAffine_BC_D64.obj
 0002:0000bd9c       $chain$10$mlib_ImageAffine_d64_3ch_bc 000000018007ad9c     mlib_ImageAffine_BC_D64.obj
 0002:0000bdd8       $chain$11$mlib_ImageAffine_d64_3ch_bc 000000018007add8     mlib_ImageAffine_BC_D64.obj
 0002:0000bde8       $chain$10$mlib_ImageAffine_d64_4ch_bc 000000018007ade8     mlib_ImageAffine_BC_D64.obj
 0002:0000be24       $chain$11$mlib_ImageAffine_d64_4ch_bc 000000018007ae24     mlib_ImageAffine_BC_D64.obj
 0002:0000be34       $unwind$mlib_ImageAffine_f32_1ch_bc 000000018007ae34     mlib_ImageAffine_BC_F32.obj
 0002:0000be48       $chain$11$mlib_ImageAffine_f32_1ch_bc 000000018007ae48     mlib_ImageAffine_BC_F32.obj
 0002:0000be88       $chain$12$mlib_ImageAffine_f32_1ch_bc 000000018007ae88     mlib_ImageAffine_BC_F32.obj
 0002:0000be98       $unwind$mlib_ImageAffine_f32_2ch_bc 000000018007ae98     mlib_ImageAffine_BC_F32.obj
 0002:0000be98       $unwind$mlib_ImageAffine_f32_3ch_bc 000000018007ae98     mlib_ImageAffine_BC_F32.obj
 0002:0000be98       $unwind$mlib_ImageAffine_f32_4ch_bc 000000018007ae98     mlib_ImageAffine_BC_F32.obj
 0002:0000beb0       $chain$10$mlib_ImageAffine_f32_2ch_bc 000000018007aeb0     mlib_ImageAffine_BC_F32.obj
 0002:0000beec       $chain$11$mlib_ImageAffine_f32_2ch_bc 000000018007aeec     mlib_ImageAffine_BC_F32.obj
 0002:0000befc       $chain$10$mlib_ImageAffine_f32_3ch_bc 000000018007aefc     mlib_ImageAffine_BC_F32.obj
 0002:0000bf38       $chain$11$mlib_ImageAffine_f32_3ch_bc 000000018007af38     mlib_ImageAffine_BC_F32.obj
 0002:0000bf48       $chain$10$mlib_ImageAffine_f32_4ch_bc 000000018007af48     mlib_ImageAffine_BC_F32.obj
 0002:0000bf84       $chain$11$mlib_ImageAffine_f32_4ch_bc 000000018007af84     mlib_ImageAffine_BC_F32.obj
 0002:0000bf94       $chain$11$mlib_ImageAffine_s32_1ch_bc 000000018007af94     mlib_ImageAffine_BC_S32.obj
 0002:0000bfd4       $chain$12$mlib_ImageAffine_s32_1ch_bc 000000018007afd4     mlib_ImageAffine_BC_S32.obj
 0002:0000bfe4       $unwind$mlib_ImageAffine_s32_2ch_bc 000000018007afe4     mlib_ImageAffine_BC_S32.obj
 0002:0000bfe4       $unwind$mlib_ImageAffine_s32_3ch_bc 000000018007afe4     mlib_ImageAffine_BC_S32.obj
 0002:0000bfe4       $unwind$mlib_ImageAffine_s32_4ch_bc 000000018007afe4     mlib_ImageAffine_BC_S32.obj
 0002:0000bff8       $chain$11$mlib_ImageAffine_s32_2ch_bc 000000018007aff8     mlib_ImageAffine_BC_S32.obj
 0002:0000c038       $chain$12$mlib_ImageAffine_s32_2ch_bc 000000018007b038     mlib_ImageAffine_BC_S32.obj
 0002:0000c048       $chain$11$mlib_ImageAffine_s32_3ch_bc 000000018007b048     mlib_ImageAffine_BC_S32.obj
 0002:0000c088       $chain$12$mlib_ImageAffine_s32_3ch_bc 000000018007b088     mlib_ImageAffine_BC_S32.obj
 0002:0000c098       $chain$11$mlib_ImageAffine_s32_4ch_bc 000000018007b098     mlib_ImageAffine_BC_S32.obj
 0002:0000c0d8       $chain$12$mlib_ImageAffine_s32_4ch_bc 000000018007b0d8     mlib_ImageAffine_BC_S32.obj
 0002:0000c0e8       $unwind$mlib_ImageAffine_d64_1ch_bl 000000018007b0e8     mlib_ImageAffine_BL_D64.obj
 0002:0000c0e8       $unwind$mlib_ImageAffine_f32_1ch_bl 000000018007b0e8     mlib_ImageAffine_BL_F32.obj
 0002:0000c100       $chain$6$mlib_ImageAffine_d64_1ch_bl 000000018007b100     mlib_ImageAffine_BL_D64.obj
 0002:0000c12c       $chain$7$mlib_ImageAffine_d64_1ch_bl 000000018007b12c     mlib_ImageAffine_BL_D64.obj
 0002:0000c13c       $unwind$mlib_ImageAffine_d64_2ch_bl 000000018007b13c     mlib_ImageAffine_BL_D64.obj
 0002:0000c13c       $unwind$mlib_ImageAffine_f32_2ch_bl 000000018007b13c     mlib_ImageAffine_BL_F32.obj
 0002:0000c150       $chain$11$mlib_ImageAffine_d64_2ch_bl 000000018007b150     mlib_ImageAffine_BL_D64.obj
 0002:0000c190       $chain$12$mlib_ImageAffine_d64_2ch_bl 000000018007b190     mlib_ImageAffine_BL_D64.obj
 0002:0000c1a0       $unwind$mlib_ImageAffine_d64_3ch_bl 000000018007b1a0     mlib_ImageAffine_BL_D64.obj
 0002:0000c1a0       $unwind$mlib_ImageAffine_f32_3ch_bl 000000018007b1a0     mlib_ImageAffine_BL_F32.obj
 0002:0000c1b4       $chain$11$mlib_ImageAffine_d64_3ch_bl 000000018007b1b4     mlib_ImageAffine_BL_D64.obj
 0002:0000c1f4       $chain$12$mlib_ImageAffine_d64_3ch_bl 000000018007b1f4     mlib_ImageAffine_BL_D64.obj
 0002:0000c204       $unwind$mlib_ImageAffine_d64_4ch_bl 000000018007b204     mlib_ImageAffine_BL_D64.obj
 0002:0000c218       $chain$11$mlib_ImageAffine_d64_4ch_bl 000000018007b218     mlib_ImageAffine_BL_D64.obj
 0002:0000c258       $chain$12$mlib_ImageAffine_d64_4ch_bl 000000018007b258     mlib_ImageAffine_BL_D64.obj
 0002:0000c268       $chain$6$mlib_ImageAffine_f32_1ch_bl 000000018007b268     mlib_ImageAffine_BL_F32.obj
 0002:0000c294       $chain$7$mlib_ImageAffine_f32_1ch_bl 000000018007b294     mlib_ImageAffine_BL_F32.obj
 0002:0000c2a4       $chain$11$mlib_ImageAffine_f32_2ch_bl 000000018007b2a4     mlib_ImageAffine_BL_F32.obj
 0002:0000c2e4       $chain$12$mlib_ImageAffine_f32_2ch_bl 000000018007b2e4     mlib_ImageAffine_BL_F32.obj
 0002:0000c2f4       $chain$11$mlib_ImageAffine_f32_3ch_bl 000000018007b2f4     mlib_ImageAffine_BL_F32.obj
 0002:0000c334       $chain$12$mlib_ImageAffine_f32_3ch_bl 000000018007b334     mlib_ImageAffine_BL_F32.obj
 0002:0000c344       $unwind$mlib_ImageAffine_f32_4ch_bl 000000018007b344     mlib_ImageAffine_BL_F32.obj
 0002:0000c358       $chain$11$mlib_ImageAffine_f32_4ch_bl 000000018007b358     mlib_ImageAffine_BL_F32.obj
 0002:0000c398       $chain$12$mlib_ImageAffine_f32_4ch_bl 000000018007b398     mlib_ImageAffine_BL_F32.obj
 0002:0000c3a8       $chain$11$mlib_ImageAffine_s32_1ch_bl 000000018007b3a8     mlib_ImageAffine_BL_S32.obj
 0002:0000c3e8       $chain$12$mlib_ImageAffine_s32_1ch_bl 000000018007b3e8     mlib_ImageAffine_BL_S32.obj
 0002:0000c3f8       $unwind$mlib_ImageAffine_s32_2ch_bl 000000018007b3f8     mlib_ImageAffine_BL_S32.obj
 0002:0000c40c       $chain$11$mlib_ImageAffine_s32_2ch_bl 000000018007b40c     mlib_ImageAffine_BL_S32.obj
 0002:0000c44c       $chain$12$mlib_ImageAffine_s32_2ch_bl 000000018007b44c     mlib_ImageAffine_BL_S32.obj
 0002:0000c45c       $unwind$mlib_ImageAffine_s32_3ch_bl 000000018007b45c     mlib_ImageAffine_BL_S32.obj
 0002:0000c470       $chain$11$mlib_ImageAffine_s32_3ch_bl 000000018007b470     mlib_ImageAffine_BL_S32.obj
 0002:0000c4b0       $chain$12$mlib_ImageAffine_s32_3ch_bl 000000018007b4b0     mlib_ImageAffine_BL_S32.obj
 0002:0000c4c0       $unwind$mlib_ImageAffine_s32_4ch_bl 000000018007b4c0     mlib_ImageAffine_BL_S32.obj
 0002:0000c4d4       $chain$11$mlib_ImageAffine_s32_4ch_bl 000000018007b4d4     mlib_ImageAffine_BL_S32.obj
 0002:0000c514       $chain$12$mlib_ImageAffine_s32_4ch_bl 000000018007b514     mlib_ImageAffine_BL_S32.obj
 0002:0000c524       $unwind$mlib_ImageAffine_s32_1ch_nn 000000018007b524     mlib_ImageAffine_NN.obj
 0002:0000c52c       $unwind$mlib_ImageAffine_d64_1ch_nn 000000018007b52c     mlib_ImageAffine_NN.obj
 0002:0000c52c       $unwind$mlib_ImageAffine_d64_2ch_nn 000000018007b52c     mlib_ImageAffine_NN.obj
 0002:0000c52c       $unwind$mlib_ImageAffine_d64_3ch_nn 000000018007b52c     mlib_ImageAffine_NN.obj
 0002:0000c52c       $unwind$mlib_ImageAffine_d64_4ch_nn 000000018007b52c     mlib_ImageAffine_NN.obj
 0002:0000c52c       $unwind$mlib_ImageAffine_s32_2ch_nn 000000018007b52c     mlib_ImageAffine_NN.obj
 0002:0000c52c       $unwind$mlib_ImageAffine_s32_3ch_nn 000000018007b52c     mlib_ImageAffine_NN.obj
 0002:0000c52c       $unwind$mlib_ImageAffine_s32_4ch_nn 000000018007b52c     mlib_ImageAffine_NN.obj
 0002:0000c534       $unwind$mlib_ImageClippingMxN 000000018007b534     mlib_ImageClipping.obj
 0002:0000c544       $chain$2$mlib_ImageClippingMxN 000000018007b544     mlib_ImageClipping.obj
 0002:0000c560       $chain$3$mlib_ImageClippingMxN 000000018007b560     mlib_ImageClipping.obj
 0002:0000c570       $unwind$mlib_ImageConvClearEdge_Bit 000000018007b570     mlib_ImageConvClearEdge_Bit.obj
 0002:0000c580       $chain$3$mlib_ImageConvClearEdge_Bit 000000018007b580     mlib_ImageConvClearEdge_Bit.obj
 0002:0000c5a0       $chain$4$mlib_ImageConvClearEdge_Bit 000000018007b5a0     mlib_ImageConvClearEdge_Bit.obj
 0002:0000c5b0       $unwind$mlib_ImageConvClearEdge_Fp 000000018007b5b0     mlib_ImageConvClearEdge_Fp.obj
 0002:0000c5c8       $unwind$mlib_ImageConvCopyEdge_Bit 000000018007b5c8     mlib_ImageConvCopyEdge_Bit.obj
 0002:0000c5e0       $unwind$j2d_mlib_ImageConvKernelConvert 000000018007b5e0     mlib_ImageConvKernelConvert.obj
 0002:0000c600       $chain$0$j2d_mlib_ImageConvKernelConvert 000000018007b600     mlib_ImageConvKernelConvert.obj
 0002:0000c614       $chain$2$j2d_mlib_ImageConvKernelConvert 000000018007b614     mlib_ImageConvKernelConvert.obj
 0002:0000c62c       $chain$3$j2d_mlib_ImageConvKernelConvert 000000018007b62c     mlib_ImageConvKernelConvert.obj
 0002:0000c63c       $chain$4$j2d_mlib_ImageConvKernelConvert 000000018007b63c     mlib_ImageConvKernelConvert.obj
 0002:0000c63c       $chain$6$j2d_mlib_ImageConvKernelConvert 000000018007b63c     mlib_ImageConvKernelConvert.obj
 0002:0000c64c       $chain$5$j2d_mlib_ImageConvKernelConvert 000000018007b64c     mlib_ImageConvKernelConvert.obj
 0002:0000c660       $unwind$mlib_ImageConvMxN_f 000000018007b660     mlib_ImageConvMxN.obj
 0002:0000c67c       $chain$0$mlib_ImageConvMxN_f 000000018007b67c     mlib_ImageConvMxN.obj
 0002:0000c690       $chain$1$mlib_ImageConvMxN_f 000000018007b690     mlib_ImageConvMxN.obj
 0002:0000c690       $chain$6$mlib_ImageConvMxN_f 000000018007b690     mlib_ImageConvMxN.obj
 0002:0000c6a0       $chain$2$mlib_ImageConvMxN_f 000000018007b6a0     mlib_ImageConvMxN.obj
 0002:0000c6b4       $chain$4$mlib_ImageConvMxN_f 000000018007b6b4     mlib_ImageConvMxN.obj
 0002:0000c6cc       $unwind$mlib_convMxNext_d64 000000018007b6cc     mlib_ImageConvMxN_Fp.obj
 0002:0000c6cc       $unwind$mlib_convMxNext_f32 000000018007b6cc     mlib_ImageConvMxN_Fp.obj
 0002:0000c6e8       $chain$0$mlib_convMxNext_f32 000000018007b6e8     mlib_ImageConvMxN_Fp.obj
 0002:0000c6fc       $chain$2$mlib_convMxNext_f32 000000018007b6fc     mlib_ImageConvMxN_Fp.obj
 0002:0000c714       $chain$3$mlib_convMxNext_f32 000000018007b714     mlib_ImageConvMxN_Fp.obj
 0002:0000c724       $chain$4$mlib_convMxNext_f32 000000018007b724     mlib_ImageConvMxN_Fp.obj
 0002:0000c734       $chain$0$mlib_convMxNext_d64 000000018007b734     mlib_ImageConvMxN_Fp.obj
 0002:0000c748       $chain$2$mlib_convMxNext_d64 000000018007b748     mlib_ImageConvMxN_Fp.obj
 0002:0000c760       $chain$3$mlib_convMxNext_d64 000000018007b760     mlib_ImageConvMxN_Fp.obj
 0002:0000c770       $chain$4$mlib_convMxNext_d64 000000018007b770     mlib_ImageConvMxN_Fp.obj
 0002:0000c780       $unwind$mlib_ImageConvMxNMulAdd_D64 000000018007b780     mlib_ImageConvMxN_Fp.obj
 0002:0000c780       $unwind$mlib_ImageConvMxNMulAdd_F32 000000018007b780     mlib_ImageConvMxN_Fp.obj
 0002:0000c7a8       $chain$1$mlib_ImageConvMxNMulAdd_F32 000000018007b7a8     mlib_ImageConvMxN_Fp.obj
 0002:0000c7c0       $chain$2$mlib_ImageConvMxNMulAdd_F32 000000018007b7c0     mlib_ImageConvMxN_Fp.obj
 0002:0000c7d0       $chain$1$mlib_ImageConvMxNMulAdd_D64 000000018007b7d0     mlib_ImageConvMxN_Fp.obj
 0002:0000c7e8       $chain$2$mlib_ImageConvMxNMulAdd_D64 000000018007b7e8     mlib_ImageConvMxN_Fp.obj
 0002:0000c7f8       $unwind$mlib_convMxNext_s32 000000018007b7f8     mlib_ImageConvMxN_ext.obj
 0002:0000c820       $chain$0$mlib_convMxNext_s32 000000018007b820     mlib_ImageConvMxN_ext.obj
 0002:0000c834       $chain$1$mlib_convMxNext_s32 000000018007b834     mlib_ImageConvMxN_ext.obj
 0002:0000c844       $unwind$mlib_ImageConvMxNMulAdd_S32 000000018007b844     mlib_ImageConvMxN_ext.obj
 0002:0000c854       $chain$8$mlib_ImageConvMxNMulAdd_S32 000000018007b854     mlib_ImageConvMxN_ext.obj
 0002:0000c888       $chain$9$mlib_ImageConvMxNMulAdd_S32 000000018007b888     mlib_ImageConvMxN_ext.obj
 0002:0000c898       $unwind$mlib_ImageConvMxNS322S32_ext 000000018007b898     mlib_ImageConvMxN_ext.obj
 0002:0000c8a0       $chain$3$mlib_ImageConvMxNS322S32_ext 000000018007b8a0     mlib_ImageConvMxN_ext.obj
 0002:0000c8c0       $chain$4$mlib_ImageConvMxNS322S32_ext 000000018007b8c0     mlib_ImageConvMxN_ext.obj
 0002:0000c8d8       $chain$5$mlib_ImageConvMxNS322S32_ext 000000018007b8d8     mlib_ImageConvMxN_ext.obj
 0002:0000c8ec       $unwind$mlib_convMxNext_s16 000000018007b8ec     mlib_ImageConv_16ext.obj
 0002:0000c8ec       $unwind$mlib_c_convMxNext_u8 000000018007b8ec     mlib_ImageConv_8ext.obj
 0002:0000c918       $chain$7$mlib_convMxNext_s16 000000018007b918     mlib_ImageConv_16ext.obj
 0002:0000c948       $chain$8$mlib_convMxNext_s16 000000018007b948     mlib_ImageConv_16ext.obj
 0002:0000c958       $unwind$mlib_i_convMxNext_s16 000000018007b958     mlib_ImageConv_16ext.obj
 0002:0000c958       $unwind$mlib_i_convMxNext_u16 000000018007b958     mlib_ImageConv_u16ext.obj
 0002:0000c984       $chain$0$mlib_i_convMxNext_s16 000000018007b984     mlib_ImageConv_16ext.obj
 0002:0000c998       $chain$1$mlib_i_convMxNext_s16 000000018007b998     mlib_ImageConv_16ext.obj
 0002:0000c9a8       $unwind$mlib_ImageConv1xN_ext 000000018007b9a8     mlib_ImageConv_16ext.obj
 0002:0000c9c8       $chain$0$mlib_ImageConv1xN_ext 000000018007b9c8     mlib_ImageConv_16ext.obj
 0002:0000c9dc       $chain$7$mlib_ImageConv1xN_ext 000000018007b9dc     mlib_ImageConv_16ext.obj
 0002:0000ca08       $chain$8$mlib_ImageConv1xN_ext 000000018007ba08     mlib_ImageConv_16ext.obj
 0002:0000ca18       $chain$11$mlib_ImageConv1xN_ext 000000018007ba18     mlib_ImageConv_16ext.obj
 0002:0000ca18       $chain$9$mlib_ImageConv1xN_ext 000000018007ba18     mlib_ImageConv_16ext.obj
 0002:0000ca28       $chain$10$mlib_ImageConv1xN_ext 000000018007ba28     mlib_ImageConv_16ext.obj
 0002:0000ca58       $unwind$mlib_i_convMxNnw_s16 000000018007ba58     mlib_ImageConv_16nw.obj
 0002:0000ca58       $unwind$mlib_i_convMxNnw_u16 000000018007ba58     mlib_ImageConv_u16nw.obj
 0002:0000ca80       $unwind$mlib_ImageConv1xN  000000018007ba80     mlib_ImageConv_16nw.obj
 0002:0000ca94       $chain$5$mlib_ImageConv1xN 000000018007ba94     mlib_ImageConv_16nw.obj
 0002:0000cabc       $chain$13$mlib_ImageConv1xN 000000018007babc     mlib_ImageConv_16nw.obj
 0002:0000caec       $chain$14$mlib_ImageConv1xN 000000018007baec     mlib_ImageConv_16nw.obj
 0002:0000cafc       $chain$15$mlib_ImageConv1xN 000000018007bafc     mlib_ImageConv_16nw.obj
 0002:0000cb0c       $unwind$mlib_convMxNnw_s16 000000018007bb0c     mlib_ImageConv_16nw.obj
 0002:0000cb3c       $chain$6$mlib_convMxNnw_s16 000000018007bb3c     mlib_ImageConv_16nw.obj
 0002:0000cb68       $chain$7$mlib_convMxNnw_s16 000000018007bb68     mlib_ImageConv_16nw.obj
 0002:0000cb78       $unwind$mlib_convMxNnw_s32 000000018007bb78     mlib_ImageConv_32nw.obj
 0002:0000cba8       $chain$6$mlib_convMxNnw_s32 000000018007bba8     mlib_ImageConv_32nw.obj
 0002:0000cbd4       $chain$7$mlib_convMxNnw_s32 000000018007bbd4     mlib_ImageConv_32nw.obj
 0002:0000cbe4       $unwind$mlib_ImageConv1xN  000000018007bbe4     mlib_ImageConv_32nw.obj
 0002:0000cbf8       $chain$6$mlib_ImageConv1xN 000000018007bbf8     mlib_ImageConv_32nw.obj
 0002:0000cc24       $chain$14$mlib_ImageConv1xN 000000018007bc24     mlib_ImageConv_32nw.obj
 0002:0000cc54       $chain$15$mlib_ImageConv1xN 000000018007bc54     mlib_ImageConv_32nw.obj
 0002:0000cc64       $chain$16$mlib_ImageConv1xN 000000018007bc64     mlib_ImageConv_32nw.obj
 0002:0000cc74       $chain$7$mlib_c_convMxNext_u8 000000018007bc74     mlib_ImageConv_8ext.obj
 0002:0000cca4       $chain$8$mlib_c_convMxNext_u8 000000018007bca4     mlib_ImageConv_8ext.obj
 0002:0000ccb4       $unwind$mlib_i_convMxNext_u8 000000018007bcb4     mlib_ImageConv_8ext.obj
 0002:0000cce0       $chain$0$mlib_i_convMxNext_u8 000000018007bce0     mlib_ImageConv_8ext.obj
 0002:0000ccf4       $chain$1$mlib_i_convMxNext_u8 000000018007bcf4     mlib_ImageConv_8ext.obj
 0002:0000cd04       $unwind$mlib_ImageConv1xN_ext 000000018007bd04     mlib_ImageConv_8ext.obj
 0002:0000cd24       $chain$0$mlib_ImageConv1xN_ext 000000018007bd24     mlib_ImageConv_8ext.obj
 0002:0000cd38       $chain$8$mlib_ImageConv1xN_ext 000000018007bd38     mlib_ImageConv_8ext.obj
 0002:0000cd68       $chain$9$mlib_ImageConv1xN_ext 000000018007bd68     mlib_ImageConv_8ext.obj
 0002:0000cd78       $chain$10$mlib_ImageConv1xN_ext 000000018007bd78     mlib_ImageConv_8ext.obj
 0002:0000cd78       $chain$12$mlib_ImageConv1xN_ext 000000018007bd78     mlib_ImageConv_8ext.obj
 0002:0000cd88       $chain$11$mlib_ImageConv1xN_ext 000000018007bd88     mlib_ImageConv_8ext.obj
 0002:0000cdbc       $unwind$mlib_c_convMxNnw_u8 000000018007bdbc     mlib_ImageConv_8nw.obj
 0002:0000cdec       $chain$6$mlib_c_convMxNnw_u8 000000018007bdec     mlib_ImageConv_8nw.obj
 0002:0000ce18       $chain$7$mlib_c_convMxNnw_u8 000000018007be18     mlib_ImageConv_8nw.obj
 0002:0000ce28       $unwind$mlib_i_convMxNnw_u8 000000018007be28     mlib_ImageConv_8nw.obj
 0002:0000ce4c       $chain$0$mlib_i_convMxNnw_u8 000000018007be4c     mlib_ImageConv_8nw.obj
 0002:0000ce60       $chain$1$mlib_i_convMxNnw_u8 000000018007be60     mlib_ImageConv_8nw.obj
 0002:0000ce70       $unwind$mlib_ImageConv1xN  000000018007be70     mlib_ImageConv_8nw.obj
 0002:0000ce84       $chain$6$mlib_ImageConv1xN 000000018007be84     mlib_ImageConv_8nw.obj
 0002:0000ceb0       $chain$14$mlib_ImageConv1xN 000000018007beb0     mlib_ImageConv_8nw.obj
 0002:0000cee0       $chain$15$mlib_ImageConv1xN 000000018007bee0     mlib_ImageConv_8nw.obj
 0002:0000cef0       $chain$16$mlib_ImageConv1xN 000000018007bef0     mlib_ImageConv_8nw.obj
 0002:0000cf00       $unwind$mlib_convMxNnw_d64 000000018007bf00     mlib_ImageConv_D64nw.obj
 0002:0000cf18       $chain$10$mlib_convMxNnw_d64 000000018007bf18     mlib_ImageConv_D64nw.obj
 0002:0000cf54       $chain$11$mlib_convMxNnw_d64 000000018007bf54     mlib_ImageConv_D64nw.obj
 0002:0000cf64       $unwind$mlib_ImageConv1xN  000000018007bf64     mlib_ImageConv_D64nw.obj
 0002:0000cf78       $chain$6$mlib_ImageConv1xN 000000018007bf78     mlib_ImageConv_D64nw.obj
 0002:0000cfa4       $chain$11$mlib_ImageConv1xN 000000018007bfa4     mlib_ImageConv_D64nw.obj
 0002:0000cfc8       $chain$12$mlib_ImageConv1xN 000000018007bfc8     mlib_ImageConv_D64nw.obj
 0002:0000cfd8       $chain$13$mlib_ImageConv1xN 000000018007bfd8     mlib_ImageConv_D64nw.obj
 0002:0000cfe8       $unwind$mlib_convMxNnw_f32 000000018007bfe8     mlib_ImageConv_F32nw.obj
 0002:0000d00c       $chain$9$mlib_convMxNnw_f32 000000018007c00c     mlib_ImageConv_F32nw.obj
 0002:0000d044       $chain$10$mlib_convMxNnw_f32 000000018007c044     mlib_ImageConv_F32nw.obj
 0002:0000d054       $chain$11$mlib_convMxNnw_f32 000000018007c054     mlib_ImageConv_F32nw.obj
 0002:0000d08c       $unwind$mlib_ImageConv1xN  000000018007c08c     mlib_ImageConv_F32nw.obj
 0002:0000d0a0       $chain$6$mlib_ImageConv1xN 000000018007c0a0     mlib_ImageConv_F32nw.obj
 0002:0000d0cc       $chain$11$mlib_ImageConv1xN 000000018007c0cc     mlib_ImageConv_F32nw.obj
 0002:0000d0f0       $chain$12$mlib_ImageConv1xN 000000018007c0f0     mlib_ImageConv_F32nw.obj
 0002:0000d100       $chain$13$mlib_ImageConv1xN 000000018007c100     mlib_ImageConv_F32nw.obj
 0002:0000d110       $unwind$mlib_convMxNext_u16 000000018007c110     mlib_ImageConv_u16ext.obj
 0002:0000d13c       $chain$7$mlib_convMxNext_u16 000000018007c13c     mlib_ImageConv_u16ext.obj
 0002:0000d16c       $chain$8$mlib_convMxNext_u16 000000018007c16c     mlib_ImageConv_u16ext.obj
 0002:0000d17c       $chain$0$mlib_i_convMxNext_u16 000000018007c17c     mlib_ImageConv_u16ext.obj
 0002:0000d190       $chain$1$mlib_i_convMxNext_u16 000000018007c190     mlib_ImageConv_u16ext.obj
 0002:0000d1a0       $unwind$mlib_ImageConv1xN_ext 000000018007c1a0     mlib_ImageConv_u16ext.obj
 0002:0000d1c0       $chain$0$mlib_ImageConv1xN_ext 000000018007c1c0     mlib_ImageConv_u16ext.obj
 0002:0000d1d4       $chain$8$mlib_ImageConv1xN_ext 000000018007c1d4     mlib_ImageConv_u16ext.obj
 0002:0000d204       $chain$9$mlib_ImageConv1xN_ext 000000018007c204     mlib_ImageConv_u16ext.obj
 0002:0000d214       $chain$10$mlib_ImageConv1xN_ext 000000018007c214     mlib_ImageConv_u16ext.obj
 0002:0000d214       $chain$12$mlib_ImageConv1xN_ext 000000018007c214     mlib_ImageConv_u16ext.obj
 0002:0000d224       $chain$11$mlib_ImageConv1xN_ext 000000018007c224     mlib_ImageConv_u16ext.obj
 0002:0000d258       $unwind$mlib_ImageConv1xN  000000018007c258     mlib_ImageConv_u16nw.obj
 0002:0000d26c       $chain$5$mlib_ImageConv1xN 000000018007c26c     mlib_ImageConv_u16nw.obj
 0002:0000d294       $chain$14$mlib_ImageConv1xN 000000018007c294     mlib_ImageConv_u16nw.obj
 0002:0000d2c8       $chain$15$mlib_ImageConv1xN 000000018007c2c8     mlib_ImageConv_u16nw.obj
 0002:0000d2d8       $chain$16$mlib_ImageConv1xN 000000018007c2d8     mlib_ImageConv_u16nw.obj
 0002:0000d2e8       $unwind$mlib_convMxNnw_u16 000000018007c2e8     mlib_ImageConv_u16nw.obj
 0002:0000d318       $chain$6$mlib_convMxNnw_u16 000000018007c318     mlib_ImageConv_u16nw.obj
 0002:0000d344       $chain$7$mlib_convMxNnw_u16 000000018007c344     mlib_ImageConv_u16nw.obj
 0002:0000d354       $unwind$mlib_ImageCopy_bit_na 000000018007c354     mlib_ImageCopy_Bit.obj
 0002:0000d35c       $chain$3$mlib_ImageCopy_bit_na 000000018007c35c     mlib_ImageCopy_Bit.obj
 0002:0000d37c       $chain$4$mlib_ImageCopy_bit_na 000000018007c37c     mlib_ImageCopy_Bit.obj
 0002:0000d38c       $unwind$j2d_mlib_ImageCreate 000000018007c38c     mlib_ImageCreate.obj
 0002:0000d3a8       $unwind$j2d_mlib_ImageCreateStruct 000000018007c3a8     mlib_ImageCreate.obj
 0002:0000d3c0       $unwind$j2d_mlib_ImageDelete 000000018007c3c0     mlib_ImageCreate.obj
 0002:0000d3c8       $unwind$mlib_ImageSet      000000018007c3c8     mlib_ImageCreate.obj
 0002:0000d3dc       $chain$0$mlib_ImageSet     000000018007c3dc     mlib_ImageCreate.obj
 0002:0000d3f0       $chain$1$mlib_ImageSet     000000018007c3f0     mlib_ImageCreate.obj
 0002:0000d400       $unwind$mlib_ImageSetSubimage 000000018007c400     mlib_ImageCreate.obj
 0002:0000d410       $chain$0$mlib_ImageSetSubimage 000000018007c410     mlib_ImageCreate.obj
 0002:0000d424       $chain$1$mlib_ImageSetSubimage 000000018007c424     mlib_ImageCreate.obj
 0002:0000d434       $unwind$mlib_ImageLookUp_U8_D64 000000018007c434     mlib_ImageLookUp_64.obj
 0002:0000d434       $unwind$mlib_c_ImageLookUpSI_U8_S32 000000018007c434     mlib_c_ImageLookUp_f.obj
 0002:0000d44c       $unwind$mlib_ImageLookUpSI_U16_D64 000000018007c44c     mlib_ImageLookUp_64.obj
 0002:0000d44c       $unwind$mlib_ImageLookUp_S16_D64 000000018007c44c     mlib_ImageLookUp_64.obj
 0002:0000d44c       $unwind$mlib_ImageLookUp_S32_D64 000000018007c44c     mlib_ImageLookUp_64.obj
 0002:0000d464       $chain$2$mlib_ImageLookUp_S16_D64 000000018007c464     mlib_ImageLookUp_64.obj
 0002:0000d480       $chain$3$mlib_ImageLookUp_S16_D64 000000018007c480     mlib_ImageLookUp_64.obj
 0002:0000d490       $unwind$mlib_ImageLookUp_U16_D64 000000018007c490     mlib_ImageLookUp_64.obj
 0002:0000d4a8       $chain$3$mlib_ImageLookUp_U16_D64 000000018007c4a8     mlib_ImageLookUp_64.obj
 0002:0000d4c8       $chain$4$mlib_ImageLookUp_U16_D64 000000018007c4c8     mlib_ImageLookUp_64.obj
 0002:0000d4d8       $chain$2$mlib_ImageLookUp_S32_D64 000000018007c4d8     mlib_ImageLookUp_64.obj
 0002:0000d4f4       $chain$3$mlib_ImageLookUp_S32_D64 000000018007c4f4     mlib_ImageLookUp_64.obj
 0002:0000d504       $unwind$mlib_ImageLookUpSI_U8_D64 000000018007c504     mlib_ImageLookUp_64.obj
 0002:0000d520       $unwind$mlib_ImageLookUpSI_S16_D64 000000018007c520     mlib_ImageLookUp_64.obj
 0002:0000d520       $unwind$mlib_ImageLookUpSI_S32_D64 000000018007c520     mlib_ImageLookUp_64.obj
 0002:0000d520       $unwind$mlib_c_ImageLookUpSI_S32_U8 000000018007c520     mlib_c_ImageLookUp_f.obj
 0002:0000d53c       $chain$1$mlib_ImageLookUpSI_S16_D64 000000018007c53c     mlib_ImageLookUp_64.obj
 0002:0000d554       $chain$2$mlib_ImageLookUpSI_S16_D64 000000018007c554     mlib_ImageLookUp_64.obj
 0002:0000d564       $chain$2$mlib_ImageLookUpSI_U16_D64 000000018007c564     mlib_ImageLookUp_64.obj
 0002:0000d580       $chain$3$mlib_ImageLookUpSI_U16_D64 000000018007c580     mlib_ImageLookUp_64.obj
 0002:0000d590       $chain$1$mlib_ImageLookUpSI_S32_D64 000000018007c590     mlib_ImageLookUp_64.obj
 0002:0000d5a8       $chain$2$mlib_ImageLookUpSI_S32_D64 000000018007c5a8     mlib_ImageLookUp_64.obj
 0002:0000d5b8       $unwind$mlib_ImageLookUp_Bit_U8_1 000000018007c5b8     mlib_ImageLookUp_Bit.obj
 0002:0000d5d8       $chain$0$mlib_ImageLookUp_Bit_U8_1 000000018007c5d8     mlib_ImageLookUp_Bit.obj
 0002:0000d5ec       $chain$1$mlib_ImageLookUp_Bit_U8_1 000000018007c5ec     mlib_ImageLookUp_Bit.obj
 0002:0000d5fc       $unwind$mlib_ImageLookUp_Bit_U8_2 000000018007c5fc     mlib_ImageLookUp_Bit.obj
 0002:0000d618       $chain$1$mlib_ImageLookUp_Bit_U8_2 000000018007c618     mlib_ImageLookUp_Bit.obj
 0002:0000d630       $chain$2$mlib_ImageLookUp_Bit_U8_2 000000018007c630     mlib_ImageLookUp_Bit.obj
 0002:0000d640       $unwind$mlib_ImageLookUp_Bit_U8_3 000000018007c640     mlib_ImageLookUp_Bit.obj
 0002:0000d65c       $chain$2$mlib_ImageLookUp_Bit_U8_3 000000018007c65c     mlib_ImageLookUp_Bit.obj
 0002:0000d678       $chain$3$mlib_ImageLookUp_Bit_U8_3 000000018007c678     mlib_ImageLookUp_Bit.obj
 0002:0000d688       $unwind$mlib_ImageLookUp_Bit_U8_4 000000018007c688     mlib_ImageLookUp_Bit.obj
 0002:0000d6a8       $chain$0$mlib_ImageLookUp_Bit_U8_4 000000018007c6a8     mlib_ImageLookUp_Bit.obj
 0002:0000d6bc       $chain$1$mlib_ImageLookUp_Bit_U8_4 000000018007c6bc     mlib_ImageLookUp_Bit.obj
 0002:0000d6cc       $unwind$mlib_AffineEdges   000000018007c6cc     mlib_ImageScanPoly.obj
 0002:0000d70c       $chain$1$mlib_AffineEdges  000000018007c70c     mlib_ImageScanPoly.obj
 0002:0000d724       $chain$2$mlib_AffineEdges  000000018007c724     mlib_ImageScanPoly.obj
 0002:0000d734       $unwind$mlib_ImageAffine_u8_1ch_bc 000000018007c734     mlib_c_ImageAffine_BC.obj
 0002:0000d744       $chain$3$mlib_ImageAffine_u8_1ch_bc 000000018007c744     mlib_c_ImageAffine_BC.obj
 0002:0000d764       $chain$4$mlib_ImageAffine_u8_1ch_bc 000000018007c764     mlib_c_ImageAffine_BC.obj
 0002:0000d774       $unwind$mlib_ImageAffine_u8_2ch_bc 000000018007c774     mlib_c_ImageAffine_BC.obj
 0002:0000d774       $unwind$mlib_ImageAffine_u8_4ch_bc 000000018007c774     mlib_c_ImageAffine_BC.obj
 0002:0000d788       $chain$2$mlib_ImageAffine_u8_2ch_bc 000000018007c788     mlib_c_ImageAffine_BC.obj
 0002:0000d7a4       $chain$3$mlib_ImageAffine_u8_2ch_bc 000000018007c7a4     mlib_c_ImageAffine_BC.obj
 0002:0000d7b4       $unwind$mlib_ImageAffine_u8_3ch_bc 000000018007c7b4     mlib_c_ImageAffine_BC.obj
 0002:0000d7c4       $chain$3$mlib_ImageAffine_u8_3ch_bc 000000018007c7c4     mlib_c_ImageAffine_BC.obj
 0002:0000d7e4       $chain$4$mlib_ImageAffine_u8_3ch_bc 000000018007c7e4     mlib_c_ImageAffine_BC.obj
 0002:0000d7f4       $chain$2$mlib_ImageAffine_u8_4ch_bc 000000018007c7f4     mlib_c_ImageAffine_BC.obj
 0002:0000d810       $chain$3$mlib_ImageAffine_u8_4ch_bc 000000018007c810     mlib_c_ImageAffine_BC.obj
 0002:0000d820       $unwind$mlib_ImageAffine_s16_1ch_bc 000000018007c820     mlib_c_ImageAffine_BC_S16.obj
 0002:0000d820       $unwind$mlib_ImageAffine_u16_1ch_bc 000000018007c820     mlib_c_ImageAffine_BC_U16.obj
 0002:0000d830       $chain$3$mlib_ImageAffine_s16_1ch_bc 000000018007c830     mlib_c_ImageAffine_BC_S16.obj
 0002:0000d850       $chain$4$mlib_ImageAffine_s16_1ch_bc 000000018007c850     mlib_c_ImageAffine_BC_S16.obj
 0002:0000d860       $unwind$mlib_ImageAffine_s16_2ch_bc 000000018007c860     mlib_c_ImageAffine_BC_S16.obj
 0002:0000d860       $unwind$mlib_ImageAffine_s16_3ch_bc 000000018007c860     mlib_c_ImageAffine_BC_S16.obj
 0002:0000d860       $unwind$mlib_ImageAffine_s16_4ch_bc 000000018007c860     mlib_c_ImageAffine_BC_S16.obj
 0002:0000d870       $chain$3$mlib_ImageAffine_s16_2ch_bc 000000018007c870     mlib_c_ImageAffine_BC_S16.obj
 0002:0000d890       $chain$4$mlib_ImageAffine_s16_2ch_bc 000000018007c890     mlib_c_ImageAffine_BC_S16.obj
 0002:0000d8a0       $chain$3$mlib_ImageAffine_s16_3ch_bc 000000018007c8a0     mlib_c_ImageAffine_BC_S16.obj
 0002:0000d8c0       $chain$4$mlib_ImageAffine_s16_3ch_bc 000000018007c8c0     mlib_c_ImageAffine_BC_S16.obj
 0002:0000d8d0       $chain$3$mlib_ImageAffine_s16_4ch_bc 000000018007c8d0     mlib_c_ImageAffine_BC_S16.obj
 0002:0000d8f0       $chain$4$mlib_ImageAffine_s16_4ch_bc 000000018007c8f0     mlib_c_ImageAffine_BC_S16.obj
 0002:0000d900       $chain$3$mlib_ImageAffine_u16_1ch_bc 000000018007c900     mlib_c_ImageAffine_BC_U16.obj
 0002:0000d920       $chain$4$mlib_ImageAffine_u16_1ch_bc 000000018007c920     mlib_c_ImageAffine_BC_U16.obj
 0002:0000d930       $unwind$mlib_ImageAffine_u16_2ch_bc 000000018007c930     mlib_c_ImageAffine_BC_U16.obj
 0002:0000d930       $unwind$mlib_ImageAffine_u16_3ch_bc 000000018007c930     mlib_c_ImageAffine_BC_U16.obj
 0002:0000d930       $unwind$mlib_ImageAffine_u16_4ch_bc 000000018007c930     mlib_c_ImageAffine_BC_U16.obj
 0002:0000d940       $chain$3$mlib_ImageAffine_u16_2ch_bc 000000018007c940     mlib_c_ImageAffine_BC_U16.obj
 0002:0000d960       $chain$4$mlib_ImageAffine_u16_2ch_bc 000000018007c960     mlib_c_ImageAffine_BC_U16.obj
 0002:0000d970       $chain$3$mlib_ImageAffine_u16_3ch_bc 000000018007c970     mlib_c_ImageAffine_BC_U16.obj
 0002:0000d990       $chain$4$mlib_ImageAffine_u16_3ch_bc 000000018007c990     mlib_c_ImageAffine_BC_U16.obj
 0002:0000d9a0       $chain$3$mlib_ImageAffine_u16_4ch_bc 000000018007c9a0     mlib_c_ImageAffine_BC_U16.obj
 0002:0000d9c0       $chain$4$mlib_ImageAffine_u16_4ch_bc 000000018007c9c0     mlib_c_ImageAffine_BC_U16.obj
 0002:0000d9d0       $unwind$mlib_ImageAffine_u8_1ch_bl 000000018007c9d0     mlib_c_ImageAffine_BL.obj
 0002:0000d9e0       $chain$2$mlib_ImageAffine_u8_1ch_bl 000000018007c9e0     mlib_c_ImageAffine_BL.obj
 0002:0000d9fc       $chain$3$mlib_ImageAffine_u8_1ch_bl 000000018007c9fc     mlib_c_ImageAffine_BL.obj
 0002:0000da0c       $unwind$mlib_ImageAffine_u8_2ch_bl 000000018007ca0c     mlib_c_ImageAffine_BL.obj
 0002:0000da20       $chain$2$mlib_ImageAffine_u8_2ch_bl 000000018007ca20     mlib_c_ImageAffine_BL.obj
 0002:0000da3c       $chain$3$mlib_ImageAffine_u8_2ch_bl 000000018007ca3c     mlib_c_ImageAffine_BL.obj
 0002:0000da4c       $unwind$mlib_ImageAffine_u8_3ch_bl 000000018007ca4c     mlib_c_ImageAffine_BL.obj
 0002:0000da60       $chain$1$mlib_ImageAffine_u8_3ch_bl 000000018007ca60     mlib_c_ImageAffine_BL.obj
 0002:0000da78       $chain$2$mlib_ImageAffine_u8_3ch_bl 000000018007ca78     mlib_c_ImageAffine_BL.obj
 0002:0000da88       $unwind$mlib_ImageAffine_u8_4ch_bl 000000018007ca88     mlib_c_ImageAffine_BL.obj
 0002:0000da9c       $chain$2$mlib_ImageAffine_u8_4ch_bl 000000018007ca9c     mlib_c_ImageAffine_BL.obj
 0002:0000dab8       $chain$3$mlib_ImageAffine_u8_4ch_bl 000000018007cab8     mlib_c_ImageAffine_BL.obj
 0002:0000dac8       $unwind$mlib_ImageAffine_s16_1ch_bl 000000018007cac8     mlib_c_ImageAffine_BL_S16.obj
 0002:0000dac8       $unwind$mlib_ImageAffine_u16_1ch_bl 000000018007cac8     mlib_c_ImageAffine_BL_U16.obj
 0002:0000dad8       $chain$2$mlib_ImageAffine_s16_1ch_bl 000000018007cad8     mlib_c_ImageAffine_BL_S16.obj
 0002:0000daf4       $chain$3$mlib_ImageAffine_s16_1ch_bl 000000018007caf4     mlib_c_ImageAffine_BL_S16.obj
 0002:0000db04       $unwind$mlib_ImageAffine_s16_2ch_bl 000000018007cb04     mlib_c_ImageAffine_BL_S16.obj
 0002:0000db04       $unwind$mlib_ImageAffine_u16_2ch_bl 000000018007cb04     mlib_c_ImageAffine_BL_U16.obj
 0002:0000db18       $chain$2$mlib_ImageAffine_s16_2ch_bl 000000018007cb18     mlib_c_ImageAffine_BL_S16.obj
 0002:0000db34       $chain$3$mlib_ImageAffine_s16_2ch_bl 000000018007cb34     mlib_c_ImageAffine_BL_S16.obj
 0002:0000db44       $unwind$mlib_ImageAffine_s16_3ch_bl 000000018007cb44     mlib_c_ImageAffine_BL_S16.obj
 0002:0000db44       $unwind$mlib_ImageAffine_u16_3ch_bl 000000018007cb44     mlib_c_ImageAffine_BL_U16.obj
 0002:0000db58       $chain$2$mlib_ImageAffine_s16_3ch_bl 000000018007cb58     mlib_c_ImageAffine_BL_S16.obj
 0002:0000db74       $chain$3$mlib_ImageAffine_s16_3ch_bl 000000018007cb74     mlib_c_ImageAffine_BL_S16.obj
 0002:0000db84       $unwind$mlib_ImageAffine_s16_4ch_bl 000000018007cb84     mlib_c_ImageAffine_BL_S16.obj
 0002:0000db84       $unwind$mlib_ImageAffine_u16_4ch_bl 000000018007cb84     mlib_c_ImageAffine_BL_U16.obj
 0002:0000db98       $chain$1$mlib_ImageAffine_s16_4ch_bl 000000018007cb98     mlib_c_ImageAffine_BL_S16.obj
 0002:0000dbb0       $chain$2$mlib_ImageAffine_s16_4ch_bl 000000018007cbb0     mlib_c_ImageAffine_BL_S16.obj
 0002:0000dbc0       $chain$2$mlib_ImageAffine_u16_1ch_bl 000000018007cbc0     mlib_c_ImageAffine_BL_U16.obj
 0002:0000dbdc       $chain$3$mlib_ImageAffine_u16_1ch_bl 000000018007cbdc     mlib_c_ImageAffine_BL_U16.obj
 0002:0000dbec       $chain$2$mlib_ImageAffine_u16_2ch_bl 000000018007cbec     mlib_c_ImageAffine_BL_U16.obj
 0002:0000dc08       $chain$3$mlib_ImageAffine_u16_2ch_bl 000000018007cc08     mlib_c_ImageAffine_BL_U16.obj
 0002:0000dc18       $chain$2$mlib_ImageAffine_u16_3ch_bl 000000018007cc18     mlib_c_ImageAffine_BL_U16.obj
 0002:0000dc34       $chain$3$mlib_ImageAffine_u16_3ch_bl 000000018007cc34     mlib_c_ImageAffine_BL_U16.obj
 0002:0000dc44       $chain$1$mlib_ImageAffine_u16_4ch_bl 000000018007cc44     mlib_c_ImageAffine_BL_U16.obj
 0002:0000dc5c       $chain$2$mlib_ImageAffine_u16_4ch_bl 000000018007cc5c     mlib_c_ImageAffine_BL_U16.obj
 0002:0000dc6c       $unwind$mlib_ImageAffine_u8_1ch_nn 000000018007cc6c     mlib_c_ImageAffine_NN.obj
 0002:0000dc84       $unwind$mlib_ImageAffine_s16_2ch_nn 000000018007cc84     mlib_c_ImageAffine_NN.obj
 0002:0000dc84       $unwind$mlib_ImageAffine_u8_2ch_nn 000000018007cc84     mlib_c_ImageAffine_NN.obj
 0002:0000dc94       $chain$2$mlib_ImageAffine_u8_2ch_nn 000000018007cc94     mlib_c_ImageAffine_NN.obj
 0002:0000dcb0       $chain$3$mlib_ImageAffine_u8_2ch_nn 000000018007ccb0     mlib_c_ImageAffine_NN.obj
 0002:0000dcc0       $unwind$mlib_ImageAffine_s16_3ch_nn 000000018007ccc0     mlib_c_ImageAffine_NN.obj
 0002:0000dcc0       $unwind$mlib_ImageAffine_u8_3ch_nn 000000018007ccc0     mlib_c_ImageAffine_NN.obj
 0002:0000dcd0       $chain$2$mlib_ImageAffine_u8_3ch_nn 000000018007ccd0     mlib_c_ImageAffine_NN.obj
 0002:0000dcec       $chain$3$mlib_ImageAffine_u8_3ch_nn 000000018007ccec     mlib_c_ImageAffine_NN.obj
 0002:0000dcfc       $unwind$mlib_ImageAffine_s16_4ch_nn 000000018007ccfc     mlib_c_ImageAffine_NN.obj
 0002:0000dcfc       $unwind$mlib_ImageAffine_u8_4ch_nn 000000018007ccfc     mlib_c_ImageAffine_NN.obj
 0002:0000dd0c       $chain$2$mlib_ImageAffine_u8_4ch_nn 000000018007cd0c     mlib_c_ImageAffine_NN.obj
 0002:0000dd28       $chain$3$mlib_ImageAffine_u8_4ch_nn 000000018007cd28     mlib_c_ImageAffine_NN.obj
 0002:0000dd38       $unwind$mlib_ImageAffine_s16_1ch_nn 000000018007cd38     mlib_c_ImageAffine_NN.obj
 0002:0000dd4c       $chain$1$mlib_ImageAffine_s16_1ch_nn 000000018007cd4c     mlib_c_ImageAffine_NN.obj
 0002:0000dd64       $chain$2$mlib_ImageAffine_s16_1ch_nn 000000018007cd64     mlib_c_ImageAffine_NN.obj
 0002:0000dd74       $chain$2$mlib_ImageAffine_s16_2ch_nn 000000018007cd74     mlib_c_ImageAffine_NN.obj
 0002:0000dd90       $chain$3$mlib_ImageAffine_s16_2ch_nn 000000018007cd90     mlib_c_ImageAffine_NN.obj
 0002:0000dda0       $chain$2$mlib_ImageAffine_s16_3ch_nn 000000018007cda0     mlib_c_ImageAffine_NN.obj
 0002:0000ddbc       $chain$3$mlib_ImageAffine_s16_3ch_nn 000000018007cdbc     mlib_c_ImageAffine_NN.obj
 0002:0000ddcc       $chain$2$mlib_ImageAffine_s16_4ch_nn 000000018007cdcc     mlib_c_ImageAffine_NN.obj
 0002:0000dde8       $chain$3$mlib_ImageAffine_s16_4ch_nn 000000018007cde8     mlib_c_ImageAffine_NN.obj
 0002:0000ddf8       $unwind$mlib_ImageConvClearEdge 000000018007cdf8     mlib_c_ImageConvClearEdge.obj
 0002:0000de08       $chain$3$mlib_ImageConvClearEdge 000000018007ce08     mlib_c_ImageConvClearEdge.obj
 0002:0000de28       $chain$5$mlib_ImageConvClearEdge 000000018007ce28     mlib_c_ImageConvClearEdge.obj
 0002:0000de48       $chain$6$mlib_ImageConvClearEdge 000000018007ce48     mlib_c_ImageConvClearEdge.obj
 0002:0000de58       $unwind$mlib_ImageConvZeroEdge 000000018007ce58     mlib_c_ImageConvClearEdge.obj
 0002:0000de68       $unwind$mlib_ImageConvCopyEdge 000000018007ce68     mlib_c_ImageConvCopyEdge.obj
 0002:0000de80       $unwind$mlib_convMxNnw_u8  000000018007ce80     mlib_c_ImageConv_f.obj
 0002:0000de98       $unwind$mlib_convMxNext_u8 000000018007ce98     mlib_c_ImageConv_f.obj
 0002:0000deb0       $unwind$mlib_ImageCopy_na  000000018007ceb0     mlib_c_ImageCopy.obj
 0002:0000deb8       $unwind$j2d_mlib_ImageLookUp 000000018007ceb8     mlib_c_ImageLookUp.obj
 0002:0000dec8       $chain$1$j2d_mlib_ImageLookUp 000000018007cec8     mlib_c_ImageLookUp.obj
 0002:0000dee0       $chain$3$j2d_mlib_ImageLookUp 000000018007cee0     mlib_c_ImageLookUp.obj
 0002:0000def8       $chain$4$j2d_mlib_ImageLookUp 000000018007cef8     mlib_c_ImageLookUp.obj
 0002:0000df08       $unwind$mlib_c_ImageLookUp_U8_S16 000000018007cf08     mlib_c_ImageLookUp_f.obj
 0002:0000df08       $unwind$mlib_c_ImageLookUp_U8_S32 000000018007cf08     mlib_c_ImageLookUp_f.obj
 0002:0000df08       $unwind$mlib_c_ImageLookUp_U8_U8 000000018007cf08     mlib_c_ImageLookUp_f.obj
 0002:0000df20       $unwind$mlib_c_ImageLookUp_S16_U8 000000018007cf20     mlib_c_ImageLookUp_f.obj
 0002:0000df38       $chain$3$mlib_c_ImageLookUp_S16_U8 000000018007cf38     mlib_c_ImageLookUp_f.obj
 0002:0000df58       $chain$4$mlib_c_ImageLookUp_S16_U8 000000018007cf58     mlib_c_ImageLookUp_f.obj
 0002:0000df68       $unwind$mlib_c_ImageLookUp_U16_U8 000000018007cf68     mlib_c_ImageLookUp_f.obj
 0002:0000df80       $chain$3$mlib_c_ImageLookUp_U16_U8 000000018007cf80     mlib_c_ImageLookUp_f.obj
 0002:0000dfa0       $chain$4$mlib_c_ImageLookUp_U16_U8 000000018007cfa0     mlib_c_ImageLookUp_f.obj
 0002:0000dfb0       $unwind$mlib_c_ImageLookUp_S32_U8 000000018007cfb0     mlib_c_ImageLookUp_f.obj
 0002:0000dfc8       $chain$3$mlib_c_ImageLookUp_S32_U8 000000018007cfc8     mlib_c_ImageLookUp_f.obj
 0002:0000dfe8       $chain$4$mlib_c_ImageLookUp_S32_U8 000000018007cfe8     mlib_c_ImageLookUp_f.obj
 0002:0000dff8       $unwind$mlib_c_ImageLookUp_S16_S16 000000018007cff8     mlib_c_ImageLookUp_f.obj
 0002:0000dff8       $unwind$mlib_c_ImageLookUp_S16_U16 000000018007cff8     mlib_c_ImageLookUp_f.obj
 0002:0000dff8       $unwind$mlib_c_ImageLookUp_S32_S32 000000018007cff8     mlib_c_ImageLookUp_f.obj
 0002:0000e010       $chain$2$mlib_c_ImageLookUp_S16_S16 000000018007d010     mlib_c_ImageLookUp_f.obj
 0002:0000e010       $chain$2$mlib_c_ImageLookUp_S16_U16 000000018007d010     mlib_c_ImageLookUp_f.obj
 0002:0000e02c       $chain$3$mlib_c_ImageLookUp_S16_S16 000000018007d02c     mlib_c_ImageLookUp_f.obj
 0002:0000e02c       $chain$3$mlib_c_ImageLookUp_S16_U16 000000018007d02c     mlib_c_ImageLookUp_f.obj
 0002:0000e03c       $unwind$mlib_c_ImageLookUp_U16_S16 000000018007d03c     mlib_c_ImageLookUp_f.obj
 0002:0000e03c       $unwind$mlib_c_ImageLookUp_U16_U16 000000018007d03c     mlib_c_ImageLookUp_f.obj
 0002:0000e058       $chain$2$mlib_c_ImageLookUp_U16_S16 000000018007d058     mlib_c_ImageLookUp_f.obj
 0002:0000e058       $chain$2$mlib_c_ImageLookUp_U16_U16 000000018007d058     mlib_c_ImageLookUp_f.obj
 0002:0000e074       $chain$3$mlib_c_ImageLookUp_U16_S16 000000018007d074     mlib_c_ImageLookUp_f.obj
 0002:0000e074       $chain$3$mlib_c_ImageLookUp_U16_U16 000000018007d074     mlib_c_ImageLookUp_f.obj
 0002:0000e084       $unwind$mlib_c_ImageLookUp_S32_S16 000000018007d084     mlib_c_ImageLookUp_f.obj
 0002:0000e084       $unwind$mlib_c_ImageLookUp_S32_U16 000000018007d084     mlib_c_ImageLookUp_f.obj
 0002:0000e09c       $chain$4$mlib_c_ImageLookUp_S32_S16 000000018007d09c     mlib_c_ImageLookUp_f.obj
 0002:0000e09c       $chain$4$mlib_c_ImageLookUp_S32_U16 000000018007d09c     mlib_c_ImageLookUp_f.obj
 0002:0000e0c0       $chain$5$mlib_c_ImageLookUp_S32_S16 000000018007d0c0     mlib_c_ImageLookUp_f.obj
 0002:0000e0c0       $chain$5$mlib_c_ImageLookUp_S32_U16 000000018007d0c0     mlib_c_ImageLookUp_f.obj
 0002:0000e0d0       $unwind$mlib_c_ImageLookUp_S16_S32 000000018007d0d0     mlib_c_ImageLookUp_f.obj
 0002:0000e0e8       $chain$3$mlib_c_ImageLookUp_S16_S32 000000018007d0e8     mlib_c_ImageLookUp_f.obj
 0002:0000e108       $chain$4$mlib_c_ImageLookUp_S16_S32 000000018007d108     mlib_c_ImageLookUp_f.obj
 0002:0000e118       $unwind$mlib_c_ImageLookUp_U16_S32 000000018007d118     mlib_c_ImageLookUp_f.obj
 0002:0000e130       $chain$3$mlib_c_ImageLookUp_U16_S32 000000018007d130     mlib_c_ImageLookUp_f.obj
 0002:0000e150       $chain$4$mlib_c_ImageLookUp_U16_S32 000000018007d150     mlib_c_ImageLookUp_f.obj
 0002:0000e160       $chain$2$mlib_c_ImageLookUp_S32_S32 000000018007d160     mlib_c_ImageLookUp_f.obj
 0002:0000e17c       $chain$3$mlib_c_ImageLookUp_S32_S32 000000018007d17c     mlib_c_ImageLookUp_f.obj
 0002:0000e18c       $unwind$mlib_c_ImageLookUpSI_U8_U8 000000018007d18c     mlib_c_ImageLookUp_f.obj
 0002:0000e1b0       $unwind$mlib_c_ImageLookUpSI_S16_U8 000000018007d1b0     mlib_c_ImageLookUp_f.obj
 0002:0000e1c0       $unwind$mlib_c_ImageLookUpSI_U16_U8 000000018007d1c0     mlib_c_ImageLookUp_f.obj
 0002:0000e1e4       $chain$1$mlib_c_ImageLookUpSI_S32_U8 000000018007d1e4     mlib_c_ImageLookUp_f.obj
 0002:0000e1fc       $chain$2$mlib_c_ImageLookUpSI_S32_U8 000000018007d1fc     mlib_c_ImageLookUp_f.obj
 0002:0000e20c       $unwind$mlib_c_ImageLookUpSI_U8_S16 000000018007d20c     mlib_c_ImageLookUp_f.obj
 0002:0000e230       $unwind$mlib_c_ImageLookUpSI_S16_S16 000000018007d230     mlib_c_ImageLookUp_f.obj
 0002:0000e230       $unwind$mlib_c_ImageLookUpSI_S16_S32 000000018007d230     mlib_c_ImageLookUp_f.obj
 0002:0000e230       $unwind$mlib_c_ImageLookUpSI_S16_U16 000000018007d230     mlib_c_ImageLookUp_f.obj
 0002:0000e230       $unwind$mlib_c_ImageLookUpSI_S32_S16 000000018007d230     mlib_c_ImageLookUp_f.obj
 0002:0000e230       $unwind$mlib_c_ImageLookUpSI_S32_S32 000000018007d230     mlib_c_ImageLookUp_f.obj
 0002:0000e230       $unwind$mlib_c_ImageLookUpSI_S32_U16 000000018007d230     mlib_c_ImageLookUp_f.obj
 0002:0000e24c       $chain$1$mlib_c_ImageLookUpSI_S16_S16 000000018007d24c     mlib_c_ImageLookUp_f.obj
 0002:0000e24c       $chain$1$mlib_c_ImageLookUpSI_S16_U16 000000018007d24c     mlib_c_ImageLookUp_f.obj
 0002:0000e264       $chain$2$mlib_c_ImageLookUpSI_S16_S16 000000018007d264     mlib_c_ImageLookUp_f.obj
 0002:0000e264       $chain$2$mlib_c_ImageLookUpSI_S16_U16 000000018007d264     mlib_c_ImageLookUp_f.obj
 0002:0000e274       $unwind$mlib_c_ImageLookUpSI_U16_S16 000000018007d274     mlib_c_ImageLookUp_f.obj
 0002:0000e274       $unwind$mlib_c_ImageLookUpSI_U16_S32 000000018007d274     mlib_c_ImageLookUp_f.obj
 0002:0000e274       $unwind$mlib_c_ImageLookUpSI_U16_U16 000000018007d274     mlib_c_ImageLookUp_f.obj
 0002:0000e290       $chain$2$mlib_c_ImageLookUpSI_U16_S16 000000018007d290     mlib_c_ImageLookUp_f.obj
 0002:0000e290       $chain$2$mlib_c_ImageLookUpSI_U16_U16 000000018007d290     mlib_c_ImageLookUp_f.obj
 0002:0000e2ac       $chain$3$mlib_c_ImageLookUpSI_U16_S16 000000018007d2ac     mlib_c_ImageLookUp_f.obj
 0002:0000e2ac       $chain$3$mlib_c_ImageLookUpSI_U16_U16 000000018007d2ac     mlib_c_ImageLookUp_f.obj
 0002:0000e2bc       $chain$1$mlib_c_ImageLookUpSI_S32_S16 000000018007d2bc     mlib_c_ImageLookUp_f.obj
 0002:0000e2bc       $chain$1$mlib_c_ImageLookUpSI_S32_U16 000000018007d2bc     mlib_c_ImageLookUp_f.obj
 0002:0000e2d4       $chain$2$mlib_c_ImageLookUpSI_S32_S16 000000018007d2d4     mlib_c_ImageLookUp_f.obj
 0002:0000e2d4       $chain$2$mlib_c_ImageLookUpSI_S32_U16 000000018007d2d4     mlib_c_ImageLookUp_f.obj
 0002:0000e2e4       $chain$1$mlib_c_ImageLookUpSI_S16_S32 000000018007d2e4     mlib_c_ImageLookUp_f.obj
 0002:0000e2fc       $chain$2$mlib_c_ImageLookUpSI_S16_S32 000000018007d2fc     mlib_c_ImageLookUp_f.obj
 0002:0000e30c       $chain$2$mlib_c_ImageLookUpSI_U16_S32 000000018007d30c     mlib_c_ImageLookUp_f.obj
 0002:0000e328       $chain$3$mlib_c_ImageLookUpSI_U16_S32 000000018007d328     mlib_c_ImageLookUp_f.obj
 0002:0000e338       $chain$1$mlib_c_ImageLookUpSI_S32_S32 000000018007d338     mlib_c_ImageLookUp_f.obj
 0002:0000e350       $chain$2$mlib_c_ImageLookUpSI_S32_S32 000000018007d350     mlib_c_ImageLookUp_f.obj
 0002:0000e360       $unwind$__GSHandlerCheckCommon 000000018007d360     MSVCRT:gshandler.obj
 0002:0000e368       $unwind$__scrt_initialize_default_local_stdio_options 000000018007d368     MSVCRT:default_local_stdio_options.obj
 0002:0000e368       $unwind$?dllmain_crt_dispatch@@YAHQEAUHINSTANCE__@@KQEAX@Z 000000018007d368     MSVCRT:dll_dllmain.obj
 0002:0000e368       $unwind$DllMain            000000018007d368     MSVCRT:dll_dllmain_stub.obj
 0002:0000e368       $unwind$__GSHandlerCheck   000000018007d368     MSVCRT:gshandler.obj
 0002:0000e368       $unwind$__scrt_acquire_startup_lock 000000018007d368     MSVCRT:utility.obj
 0002:0000e368       $unwind$__scrt_dllmain_after_initialize_c 000000018007d368     MSVCRT:utility.obj
 0002:0000e368       $unwind$__scrt_dllmain_before_initialize_c 000000018007d368     MSVCRT:utility.obj
 0002:0000e368       $unwind$__scrt_dllmain_crt_thread_attach 000000018007d368     MSVCRT:utility.obj
 0002:0000e368       $unwind$__scrt_dllmain_crt_thread_detach 000000018007d368     MSVCRT:utility.obj
 0002:0000e368       $unwind$__scrt_dllmain_uninitialize_c 000000018007d368     MSVCRT:utility.obj
 0002:0000e368       $unwind$__scrt_dllmain_uninitialize_critical 000000018007d368     MSVCRT:utility.obj
 0002:0000e370       $xdatasym                  000000018007d370     MSVCRT:amdsecgs.obj
 0002:0000e378       $xdatasym                  000000018007d378     MSVCRT:chkstk.obj
 0002:0000e380       $unwind$__isa_available_init 000000018007d380     MSVCRT:cpu_disp.obj
 0002:0000e390       $unwind$?dllmain_crt_process_attach@@YAHQEAUHINSTANCE__@@QEAX@Z 000000018007d390     MSVCRT:dll_dllmain.obj
 0002:0000e3cc       $unwind$?fin$0@?0??dllmain_crt_process_attach@@YAHQEAUHINSTANCE__@@QEAX@Z@4HA 000000018007d3cc     MSVCRT:dll_dllmain.obj
 0002:0000e3cc       $unwind$?fin$0@?0??dllmain_crt_process_detach@@YAH_N@Z@4HA 000000018007d3cc     MSVCRT:dll_dllmain.obj
 0002:0000e3cc       $unwind$?fin$1@?0??dllmain_crt_process_detach@@YAH_N@Z@4HA 000000018007d3cc     MSVCRT:dll_dllmain.obj
 0002:0000e3d4       $unwind$?dllmain_crt_process_detach@@YAH_N@Z 000000018007d3d4     MSVCRT:dll_dllmain.obj
 0002:0000e428       $unwind$?dllmain_dispatch@@YAHQEAUHINSTANCE__@@KQEAX@Z 000000018007d428     MSVCRT:dll_dllmain.obj
 0002:0000e450       $unwind$?filt$0@?0??dllmain_dispatch@@YAHQEAUHINSTANCE__@@KQEAX@Z@4HA 000000018007d450     MSVCRT:dll_dllmain.obj
 0002:0000e458       $unwind$_DllMainCRTStartup 000000018007d458     MSVCRT:dll_dllmain.obj
 0002:0000e468       $unwind$__report_gsfailure 000000018007d468     MSVCRT:gs_report.obj
 0002:0000e470       $unwind$capture_previous_context 000000018007d470     MSVCRT:gs_report.obj
 0002:0000e47c       $unwind$__raise_securityfailure 000000018007d47c     MSVCRT:gs_report.obj
 0002:0000e47c       $unwind$__scrt_initialize_crt 000000018007d47c     MSVCRT:utility.obj
 0002:0000e47c       $unwind$__scrt_initialize_onexit_tables 000000018007d47c     MSVCRT:utility.obj
 0002:0000e47c       $unwind$__scrt_release_startup_lock 000000018007d47c     MSVCRT:utility.obj
 0002:0000e47c       $unwind$__scrt_uninitialize_crt 000000018007d47c     MSVCRT:utility.obj
 0002:0000e484       $unwind$__security_init_cookie 000000018007d484     MSVCRT:gs_support.obj
 0002:0000e490       $unwind$__scrt_is_nonwritable_in_current_image 000000018007d490     MSVCRT:utility.obj
 0002:0000e4b0       $unwind$__scrt_is_nonwritable_in_current_image$filt$0 000000018007d4b0     MSVCRT:utility.obj
 0002:0000e4b8       $unwind$__scrt_dllmain_exception_filter 000000018007d4b8     MSVCRT:utility.obj
 0002:0000e4cc       $unwind$__scrt_fastfail    000000018007d4cc     MSVCRT:utility_desktop.obj
 0002:0000e4dc       $unwind$_RTC_Initialize    000000018007d4dc     MSVCRT:initsect.obj
 0002:0000e4dc       $unwind$_RTC_Terminate     000000018007d4dc     MSVCRT:initsect.obj
 0002:0000e4e8       $xdatasym                  000000018007d4e8     MSVCRT:guard_dispatch.obj
 0002:0000e4f0       $xdatasym                  000000018007d4f0     MSVCRT:guard_xfg_dispatch.obj
 0002:0000e500       .edata                     000000018007d500     mlib_image.exp
 0002:0000e528       rgpv                       000000018007d528     mlib_image.exp
 0002:0000e544       rgszName                   000000018007d544     mlib_image.exp
 0002:0000e560       rgwOrd                     000000018007d560     mlib_image.exp
 0002:0000e56e       szName                     000000018007d56e     mlib_image.exp
 0002:0000e57d       $N00001                    000000018007d57d     mlib_image.exp
 0002:0000e592       $N00002                    000000018007d592     mlib_image.exp
 0002:0000e5b2       $N00003                    000000018007d5b2     mlib_image.exp
 0002:0000e5c8       $N00004                    000000018007d5c8     mlib_image.exp
 0002:0000e5dd       $N00005                    000000018007d5dd     mlib_image.exp
 0002:0000e5f8       $N00006                    000000018007d5f8     mlib_image.exp
 0002:0000e60d       $N00007                    000000018007d60d     mlib_image.exp
 0002:0000e8f6       .idata$6                   000000018007d8f6     kernel32:KERNEL32.dll
 0002:0000e950       .idata$6                   000000018007d950     vcruntime:VCRUNTIME140.dll
 0002:0000ea1a       .idata$6                   000000018007da1a     ucrt:api-ms-win-crt-heap-l1-1-0.dll
 0002:0000ea3a       .idata$6                   000000018007da3a     ucrt:api-ms-win-crt-runtime-l1-1-0.dll
 0003:00000054       ?__proc_attached@@3HA      000000018007e054     MSVCRT:dll_dllmain.obj
 0003:00000060       GS_ExceptionRecord         000000018007e060     MSVCRT:gs_report.obj
 0003:00000100       GS_ContextRecord           000000018007e100     MSVCRT:gs_report.obj
 0003:00000600       ?is_initialized_as_dll@@3_NA 000000018007e600     MSVCRT:utility.obj
 0003:00000601       ?module_local_atexit_table_initialized@@3_NA 000000018007e601     MSVCRT:utility.obj
 0003:00000608       ?module_local_atexit_table@@3U_onexit_table_t@@A 000000018007e608     MSVCRT:utility.obj
 0003:00000620       ?module_local_at_quick_exit_table@@3U_onexit_table_t@@A 000000018007e620     MSVCRT:utility.obj
 0005:00000060       $R000000                   0000000180081060     mlib_image.dll.res
